:100000000C9407080C942F080C942F080C942F08BC
:100010000C942F080C942F080C942F080C942F0884
:100020000C942F080C942F080C942F080C942F0874
:100030000C942F080C94253B0C942F080C942F083B
:100040000C942F080C94634C0C94BD210C942F0835
:100050000C947A230C942F080C942F080C942F08DE
:10006000FEC70000FCC70000FAC70000F8C7000088
:10007000084AD73B3BCE016E84BCBFFDC12F3D6C0F
:1000800074319ABD56833DDA3D00C77F11BED9E475
:10009000BB4C3E916BAAAABE000000803F05A84C55
:1000A000CDB2D44EB93836A9020C50B99186880821
:1000B0003CA6AAAA2ABE000000803F4572726F7259
:1000C0003A005072696E7465722073746F70706557
:1000D000642064657520746F206572726F72732E70
:1000E0002046697820746865206572726F7220619D
:1000F0006E6420757365204D39393920746F207214
:10010000657374617274212E202854656D70657258
:1001100061747572652069732072657365742E2031
:10012000536574206974206265666F72652072651C
:100130007374617274696E6729005072696E7465B8
:10014000722068616C7465642E206B696C6C282960
:100150002063616C6C6564202121006F6B00526527
:1001600073656E643A006563686F3A002200556EED
:100170006B6E6F776E20636F6D6D616E643A2200F7
:100180007A5F6D696E3A00795F6D696E3A00785FEB
:100190006D696E3A005A3A00593A0020436F756E05
:1001A0007420583A00453A005A3A00593A00583AF1
:1001B000004649524D574152455F4E414D453A4DDB
:1001C00061726C696E2056313B20537072696E7497
:1001D00065722F6772626C206D617368757020663E
:1001E0006F722067656E36204649524D5741524521
:1001F0005F55524C3A687474703A2F2F7777772E88
:100200006D656E64656C2D70617274732E636F6DB5
:100210002050524F544F434F4C5F56455253494F15
:100220004E3A312E30204D414348494E455F545996
:1002300050453A4D656E64656C204558545255449E
:1002400045525F434F554E543A310A0020423A001E
:1002500020453A00543A0020573A0020453A0054CD
:100260003A0020403A00202F0020423A00202F0080
:100270006F6B20543A005072696E7465722073740B
:100280006F707065642064657520746F206572728C
:100290006F72732E204669782074686520657272CB
:1002A0006F7220616E6420757365204D3939392075
:1002B000746F2072657374617274212E20285465E6
:1002C0006D706572617475726520697320726573F3
:1002D00065742E20536574206974206265666F72A0
:1002E000652072657374617274696E6729006F6B43
:1002F000004E6F204C696E65204E756D62657220F0
:100300007769746820636865636B73756D2C204C26
:10031000617374204C696E653A004E6F20436865C6
:10032000636B73756D2077697468206C696E6520E6
:100330006E756D6265722C204C617374204C696E11
:10034000653A00636865636B73756D206D69736DE5
:10035000617463682C204C617374204C696E653A3B
:10036000004C696E65204E756D6265722069732060
:100370006E6F74204C617374204C696E65204E75ED
:100380006D6265722B312C204C617374204C696E48
:10039000653A002020506C616E6E6572427566662B
:1003A000657242797465733A200020467265652053
:1003B0004D656D6F72793A20006572696B00207C23
:1003C00020417574686F723A2000323031322D301E
:1003D000352D303200204C61737420557064617487
:1003E00065643A2000312E302E3020524332004DC9
:1003F00061726C696E3A200020536F667477617287
:100400006520526573657400205761746368646F7A
:1004100067205265736574002042726F776E206F9B
:100420007574205265736574002045787465726E2A
:10043000616C20526573657400506F7765725570FA
:10044000007374617274002200656E717565696E67
:1004500067202200002124272A002225282B0020A3
:1004600023262902020202020202020404040404F6
:100470000404040303030303030303010101010153
:10048000010101010204081020408001020408104B
:100490002040800102040810204080804020100885
:1004A000040201000000010200000000000000043E
:1004B000030706000000000000000000000000002C
:1004C0000000006563686F3A0020746F6F206C6FE6
:1004D0006E6720657874727573696F6E20707265CF
:1004E00076656E7465640020636F6C642065787453
:1004F000727573696F6E2070726576656E7465646F
:100500000024F427D3FD204D0FB0119A05160CE9F5
:10051000022D09C801650733013206DE005405A724
:1005200000AD0483002A046900C10356006B034830
:100530000023033D00E6023500B1022D00840228AD
:10054000005C0223003902200019021C00FD011981
:1005500000E4011700CD011500B8011300A5011139
:10056000009401100084010F0075010E0067010D59
:10057000005A010C004E010B0043010A0039010A28
:10058000002F010900260109001D010800150107BF
:10059000000E01080006010700FF000600F9000632
:1005A00000F3000600ED000600E7000500E200058C
:1005B00000DD000500D8000500D3000400CF0005D1
:1005C00000CA000400C6000400C2000400BE00030C
:1005D00000BB000400B7000300B4000300B1000436
:1005E00000AD000300AA000300A7000200A500035D
:1005F00000A20003009F0002009D0003009A000279
:100600000098000300950002009300020091000290
:10061000008F0002008D0002008B000200890002A2
:1006200000870002008500020083000200810001B3
:1006300000800002007E0002007C0001007B0002BE
:1006400000790001007800020076000100750001C9
:1006500000740002007200010071000100700002CD
:10066000006E0001006D0001006C0001006B0002D3
:1006700000690001006800010067000100660001D8
:1006800000650001006400010063000100620001D8
:100690000061000100600001005F0001005E0001D8
:1006A000005D0001005C0001005B0000005B0001D8
:1006B000005A0001005900010058000100570000D5
:1006C00000570001005600010055000100540000D1
:1006D00000540001005300010052000100510000CD
:1006E0000051000100500001004F0000004F0001C8
:1006F000004E0000004E0001004D0001004C0000C3
:10070000004C0001004B0000004B0001004A0001BA
:1007100000490000004900010048000000480001B5
:1007200000470000004700010046000000460001AD
:1007300000450000004500010044000000440001A5
:10074000004300000043000100420000004200019D
:100750000041000000410000004100010040000095
:1007600000400001003F0000003F0001003E00008B
:10077000003E0000003E0001003D0000003D000181
:10078000003C0000003C0000003C0001003B000079
:10079000003B0000003B0001003A0000003A00006E
:1007A000003A000100390000003900000039000162
:1007B0000038000000380000003800010037000059
:1007C000003700000037000100360000003600004E
:1007D0000036000100350000003500000035000043
:1007E0000035000100340000003400000034000136
:1007F000003300000033000000330000003300012C
:10080000003200000032000000320000003200011F
:100810000031000000310000003100000031000113
:100820000030000000300000003000000030000107
:10083000002F0000002F0000002F0000002F0001FB
:10084000002E0000002E0000002E0000002E0000F0
:10085000002E0001002D0000002D0000002D0000E2
:10086000002D0001002C0000002C0000002C0000D6
:10087000002C0000002C0001002B0000002B0000C9
:10088000002B0000002B0000002B0001002A0000BC
:10089000002A0000002A0000002A0000002A0000B0
:1008A000002A0001002900000029000000290000A2
:1008B0000029000000290000002900010028000094
:1008C0000028000000280000002800000028000187
:1008D000002700000027000000270000002700007C
:1008E000002700000027000000270001002600006C
:1008F0000026000000260000002600000026000060
:100900000024F4B12873CB111D62AECC159698F477
:1009100010A287900D127A190BF96E4009B965D3B0
:1009200007E65DB5063157D005615116054B4C7D84
:1009300004CE47FD03D14392033F403603093DE90E
:1009400002203AA4027C376A0212353602DC3208F1
:1009500002D430E101F32EBD01362D9E01982B818A
:1009600001172A6701B028500160273B012526287E
:1009700001FD241601E7230701E022F800E821EB3E
:1009800000FD20DE001F20D3004C1FC800841EBFC6
:1009900000C51DB500101DAD00631CA500BE1B9E4B
:1009A00000201B9700891A9100F8198A006E19859A
:1009B00000E9187F006A187B00EF1776007917713D
:1009C0000008176D009B166A0031166500CC156291
:1009D000006A155F000B155B00B0145800581456E0
:1009E0000002145200B013500060134E0012134B5B
:1009F00000C71249007E12460038124500F3114329
:100A000000B011400070113F0031113D00F4103C66
:100A100000B8103A007E103800461037000F10352D
:100A200000DA0F3400A60F3300730F3100420F308D
:100A300000120F3000E20E2D00B50E2D00880E2C96
:100A4000005C0E2B00310E2A00070E2800DF0D2857
:100A500000B70D2700900D26006A0D2600440D24D6
:100A600000200D2400FC0C2300D90C2200B70C221E
:100A700000950C2100740C2000540C1F00350C1F35
:100A800000160C1F00F70B1E00D90B1D00BC0B1C21
:100A900000A00B1C00840B1C00680B1B004D0B1BE3
:100AA00000320B1A00180B1900FF0A1900E60A1988
:100AB00000CD0A1800B50A18009D0A1800850A170B
:100AC000006E0A1600580A1600420A16002C0A1672
:100AD00000160A1500010A1500EC091400D80914C3
:100AE00000C4091400B00914009C091300890913FB
:100AF000007609130063091200510912003F091220
:100B0000002D0911001C0912000A091100F9081032
:100B100000E9081100D8081000C8081000B8081033
:100B200000A808100098080F0089080F007A080F25
:100B3000006B080F005C080F004D080E003F080E08
:100B40000031080E0023080E0015080E0007080DDE
:100B500000FA070D00ED070D00E0070D00D3070DAB
:100B600000C6070D00B9070C00AD070C00A1070D6A
:100B70000094070B0089070C007D070C0071070C1F
:100B80000065070B005A070B004F070B0044070BCB
:100B90000039070B002E070B0023070B0018070A6C
:100BA000000E070B0003070A00F9060A00EF060A09
:100BB00000E5060A00DB060A00D1060900C8060A9D
:100BC00000BE060900B5060A00AB060900A2060928
:100BD000009906090090060900870609007E0609AB
:100BE00000750609006C060800640609005B06082B
:100BF00000530609004A060800420608003A0608A3
:100C000000320608002A060800220608001A060814
:100C100000120607000B06080003060800FB050784
:100C200000F4050800EC050700E5050700DE0507F0
:100C300000D7050700D0050700C9050700C2050752
:100C400000BB050700B4050700AD050700A60506B3
:100C500000A005070099050700920506008C05060F
:100C600000860507007F0506007905060073050765
:100C7000006C05060066050600600506005A0506BC
:100C800000540506004E050600480506004205050D
:100C9000003D05060037050600310505002C050658
:100CA0000026050500210506001B050500160506A2
:100CB00000100505000B05050006050600000505EA
:100CC00000FB040500F6040500F1040500EC040532
:100CD00000E7040500E2040500DD040500D8040572
:100CE00000D3040500CE040500C9040500C40405B2
:100CF00000BF040400BB040500B6040500B10405F0
:100D0000006563686F3A00205A3A0020593A002083
:100D1000583A00656E6473746F7073206869743A32
:100D200020004572726F723A0054656D7065726191
:100D300074757265206865617465642062656420FD
:100D40007377697463686564206F66662E204D4111
:100D50005854454D50207472696767657265642008
:100D60002121003A2045787472756465722073778A
:100D7000697463686564206F66662E204D494E5421
:100D8000454D502074726967676572656420210063
:100D90003A2045787472756465722073776974635C
:100DA000686564206F66662E204D415854454D504D
:100DB000207472696767657265642021001000C93C
:100DC0000220013C0130020A014003EF005004DD23
:100DD000006005D0007006C5008007BC009008B513
:100DE00000A009AE00B00AA900C00BA300D00C9F60
:100DF00000E00D9A00F00E96000010930010118F85
:100E00000020128C00301388004014850050158299
:100E1000006016800070177D0080187A00901978A5
:100E200000A01A7500B01B7300C01C7000D01D6EAE
:100E300000E01E6C00F01F6A0000216700102265B0
:100E400000202363003024610040255F0050265CB1
:100E50000060275A007028580080295600902A54B4
:100E600000A02B5100B02C4F00C02D4D00D02E4BB8
:100E700000E02F4800F030460000324300103340BD
:100E80000020343D0030353A0040363700503734CA
:100E9000006038300070392C00803A2800903B22E6
:100EA00000A03C1C00B03D1400C03E0800D03F0034
:100EB00000202D20496E76616C696420657874721B
:100EC00075646572206E756D626572202100202D3B
:100ED00020496E76616C696420657874727564650A
:100EE00072206E756D626572210050494420417513
:100EF000746F74756E652066696E697368656420C9
:100F00002120506C61636520746865204B702C2033
:100F10004B6920616E64204B6420636F6E73746153
:100F20006E747320696E2074686520636F6E6669E5
:100F30006775726174696F6E2E6800504944204174
:100F400075746F74756E65206661696C65642120C7
:100F500074696D656F75740020403A006F6B2054A2
:100F60003A00504944204175746F74756E6520666F
:100F700061696C6564212054656D7065726174757A
:100F8000726520746F206869676800204B643A209E
:100F900000204B693A2000204B703A200020436C1F
:100FA000617369632050494420002054753A200041
:100FB000204B753A2000206D61783A2000206D6941
:100FC0006E3A200020643A200020626961733A2062
:100FD00000494E46494E4954594E414ECDCCCC3D28
:100FE0000AD7233C17B7D13877CC2B329595E62416
:100FF0001FB14F0A000020410000C84200401C46BB
:1010000020BCBE4CCA1B0E5AAEC59D749725112438
:101010001FBECFEFD0E1DEBFCDBF12E0A0E0B1E058
:10102000E4EFF0EB02C005900D92A438B107D9F7B8
:101030001AE0A4E8B2E001C01D92A53FB107E1F7B4
:1010400010E1CEE0D0E104C02297FE010E94C6521A
:10105000CC30D107C9F70E94B8210C9478580C9471
:101060000000AF92BF92CF92DF92EF92FF920F9368
:101070001F93DF93CF93CDB7DEB7E0970FB6F89409
:10108000DEBF0FBECDBFDE011196EFE6F2E080E1DC
:1010900001900D928150E1F7DE015196EFE5F2E00B
:1010A00080E101900D928150E1F7DE019196EFE42D
:1010B000F2E080E101900D928150E1F7BE016F5F97
:1010C0007F4F4EE155E021E1A22EB12CAC0EBD1EAA
:1010D0000EE015E091E2E92EF12CEC0EFD1E8EE201
:1010E000C82E85E0D82E20E030E0FB01819191915F
:1010F000A191B191BF01FA0181939193A193B19311
:10110000AF01F50181919191A191B1915F01F80138
:1011100081939193A193B1938F01F7018191919163
:10112000A191B1917F01F60181939193A193B19324
:101130006F012F5F3F4F24303105B9F680E090E01A
:10114000AAEFB3E48093420590934305A09344052E
:10115000B093450580E090E8ABE3B5E480934605A5
:1011600090934705A0934805B093490580E090E02F
:10117000DC0180933E0590933F05A0934005B0931A
:10118000410520E23EE440E050E020930A05309320
:101190000B0540930C0550930D05809356059093D5
:1011A0005705A0935805B093590580E090E0A0EA58
:1011B000B1E480934A0590934B05A0934C05B093FE
:1011C0004D058DEC9CECACECBEE380934E0590930A
:1011D0004F05A0935005B093510580E090E0A0EA40
:1011E000B0E48093520590935305A0935405B093B7
:1011F0005505E6E6F1E007C09091C00095FFFCCFF1
:101200008093C600319684918823B1F7E0E0F1E045
:1012100006C09091C00095FFFCCF8093C6008191DD
:101220008823B9F78091C00085FFFCCF8AE08093C6
:10123000C600E0960FB6F894DEBF0FBECDBFCF91CB
:10124000DF911F910F91FF90EF90DF90CF90BF90B3
:10125000AF900895DF93CF9300D0CDB7DEB78091E4
:10126000EF0A9091F00A9E012F5F3F4F009719F40B
:10127000255F3A4002C0281B390B3A8329838981B4
:101280009A810F900F90CF91DF910895AF92BF9206
:10129000CF92DF92EF92FF920F931F93CF93DF9342
:1012A00089E095E040E052EC61E070E00E94AF23FD
:1012B000E1E4F4E007C09091C00095FFFCCF80937B
:1012C000C600319684918823B1F78091C00085FFD4
:1012D000FCCF8AE08093C60086E691E0FC0107C05F
:1012E0003091C00035FFFCCF2093C6003196249189
:1012F0002223B1F724B720FF14C0E9E3F4E007C0CC
:101300004091C00045FFFCCF3093C6003196349128
:101310003323B1F73091C00035FFFCCF3AE0309372
:10132000C60021FF14C0E9E2F4E007C04091C0000C
:1013300045FFFCCF3093C600319634913323B1F78B
:101340003091C00035FFFCCF3AE03093C60022FF59
:1013500014C0E8E1F4E007C04091C00045FFFCCFB5
:101360003093C600319634913323B1F73091C000E9
:1013700035FFFCCF3AE03093C60023FF14C0E8E00D
:10138000F4E007C04091C00045FFFCCF3093C60099
:10139000319634913323B1F73091C00035FFFCCF43
:1013A0003AE03093C60025FF14C0E8EFF3E007C031
:1013B0003091C00035FFFCCF2093C60031962491B8
:1013C0002223B1F72091C00025FFFCCF2AE0209313
:1013D000C60014BEEFEEF3E007C03091C00035FF49
:1013E000FCCF2093C600319624912223B1F7E5EE7D
:1013F000F3E007C03091C00035FFFCCF2093C6005A
:10140000319624912223B1F72091C00025FFFCCF13
:101410002AE02093C600FC012491E6E6F1E008C032
:101420003091C00035FFFCCF2093C6003196249147
:101430002223B1F7E5EDF3E007C03091C00035FF9E
:10144000FCCF2093C600319624912223B1F7EAEC19
:10145000F3E007C03091C00035FFFCCF2093C600F9
:10146000319624912223B1F7EEEBF3E007C03091DF
:10147000C00035FFFCCF2093C60031962491222373
:10148000B1F7E9EBF3E007C03091C00035FFFCCFC6
:101490002093C600319624912223B1F72091C000F9
:1014A00025FFFCCF2AE02093C600FC018491E6E6EC
:1014B000F1E008C09091C00095FFFCCF8093C6007A
:1014C000319684918823B1F7EAEAF3E007C090915E
:1014D000C00095FFFCCF8093C6003196849188238D
:1014E000B1F7B8DEBC0189E095E04AE050E00E9427
:1014F000BC24E3E9F3E007C09091C00095FFFCCF66
:101500008093C600319684918823B1F789E095E0F5
:1015100060ED74E04AE050E00E94BC248091C0007D
:1015200085FFFCCF8AE08093C6001092720410926F
:101530007304109274041092750480E092DDCEE280
:10154000D5E00EE115E03AE5E32E35E0F32E6991A2
:10155000799189919991F801A190B190C190D19020
:101560008F010E94464FA60195010E947B510E9467
:101570001A4FF70161937193819391937F01F5E085
:10158000CE33DF0721F70E949F460E94DC2D0E9488
:101590002C41DF91CF911F910F91FF90EF90DF9041
:1015A000CF90BF90AF90089580916A0490916B04A2
:1015B000019660E070E00C94CA5280916A049091A8
:1015C0006B04019660E070E04AE050E00C94375400
:1015D000682FE091E802F091E90240E650E0E49FD4
:1015E0009001E59F300DF49F300D1124C901865103
:1015F0009D4F70E00E9481559C0190936B048093F5
:101600006A0481E02115310509F480E008950E9403
:1016100002226093B2027093B3028093B40290935B
:10162000B502EBE5F1E007C09091C00095FFFCCF5B
:101630008093C600319684918823B1F78091C000D1
:1016400085FFFCCF8AE08093C600089589E095E08D
:101650000E94F223EEE5F1E007C09091C00095FFF3
:10166000FCCF8093C600319684918823B1F74091D6
:10167000AA025091AB026091AC027091AD024F5F33
:101680005F4F6F4F7F4F89E095E02AE030E00E9486
:101690008C248091C00085FFFCCF8AE08093C60037
:1016A000B6CF4F925F926F927F928F929F92AF923E
:1016B000BF92CF92DF92EF92FF920F931F93CF933F
:1016C000DF9370E6C72ED12C64E0662E712C51E0BA
:1016D000A52EB12CE6E7F2E084904AE0942EEEEEDF
:1016E000F2E05490442443941CC28D3071F08A334C
:1016F00021F490916D04992341F020916E04309172
:101700006F042F3531050CF4EEC1E0916E04F091B9
:101710006F04309719F410926D0422C28091700406
:10172000909171048C9DE0018D9DD00D9C9DD00DFC
:101730001124EC0FFD1FE651FD4F108220916D0426
:10174000222309F0CBC110926D048E589B4FFC01EF
:1017500010828E0106511D4FC8016EE470E00E9498
:101760008155009709F412C190936B0480936A0429
:101770009501201B310B280F391F2C0F3D1FC9016C
:1017800086519D4F60E070E04AE050E00E9437547F
:10179000609376047093770480937804909379042F
:1017A000E090AA02F090AB020091AC021091AD0261
:1017B000A80197012F5F3F4F4F4F5F4F621773078D
:1017C0008407950709F43AC02091700430917104A0
:1017D0002C9DC0012D9D900D3C9D900D1124865196
:1017E0009D4F68E171E00E948C55009739F5EBEB55
:1017F000F0E007C09091C00095FFFCCF8093C60039
:10180000319684918823B1F7E1E6F3E007C0909127
:10181000C00095FFFCCF8093C60031968491882349
:10182000B1F789E095E0B801A7012AE030E00E9415
:101830008C248091C00085FFFCCF92C08091700401
:10184000909171048C9DE0018D9DD00D9C9DD00DDB
:101850001124CE0186519D4F6AE270E00E948155AD
:10186000009709F457C020E000E002C003272F5F73
:10187000FE01E20FF11DE651FD4F30813A32B1F722
:1018800090936B0480936A049E0126513D4FA501FD
:10189000421B530B9A01280F391F2C0F3D1FC90102
:1018A00086519D4F60E070E00E94CA520E94154F21
:1018B00010E00617170709F458C0EBEBF0E007C07B
:1018C0009091C00095FFFCCF8093C6003196849123
:1018D0008823B1F7E3E4F3E007C09091C00095FFDF
:1018E000FCCF8093C600319684918823B1F7409154
:1018F000AA025091AB026091AC027091AD0289E0F6
:1019000095E02AE030E00E948C248091C00085FFA1
:10191000FCCF26C0EBEBF0E007C09091C00095FF34
:10192000FCCF8093C600319684918823B1F7EAE119
:10193000F3E007C09091C00095FFFCCF8093C600F4
:10194000319684918823B1F789E095E0B801A70129
:101950002AE030E00E948C248091C00085FFFCCFFB
:101960008AE08093C60072DE47C080917604909131
:101970007704A0917804B09179048093AA0290939F
:10198000AB02A093AC02B093AD023BC0C8016AE2C7
:1019900070E00E9481550097A1F1EBEBF0E007C0E9
:1019A0009091C00095FFFCCF8093C6003196849142
:1019B0008823B1F7E1EFF2E007C09091C00095FFF6
:1019C000FCCF8093C600319684918823B1F7409173
:1019D000AA025091AB026091AC027091AD0289E015
:1019E00095E02AE030E00E948C248091C00085FFC1
:1019F000FCCF8AE08093C60010926F0410926E04B0
:101A0000AFC080917004909171048C9D80018D9D78
:101A1000100D9C9D100D1124E801C651DD4FCE0123
:101A200067E470E00E948155009709F442C09093EA
:101A30006B0480936A0495012C1B3D0B280F391F02
:101A4000200F311FC90186519D4F60E070E00E9458
:101A5000CA520E94154F6430710558F58091A90251
:101A6000882399F4852DEEEEF2E008C09091C00035
:101A700095FFFCCF8093C600319684918823B1F7FF
:101A80008091C00085FFFCCF12C0882DE6E7F2E010
:101A900008C09091C00095FFFCCF8093C60031969E
:101AA00084918823B1F78091C00085FFFCCF90928C
:101AB000C60080917004909171040196B3010E9458
:101AC0006052909371048093700480917A04909195
:101AD0007B04019690937B0480937A0410926F04A8
:101AE00010926E041EC08B3311F440926D049091DD
:101AF0006D049923B1F440917004509171044C9D90
:101B0000F0014D9DF00D5C9DF00D1124E20FF31FCF
:101B1000E651FD4F80832F5F3F4F30936F0420933A
:101B20006E0480910505909106052091070530917E
:101B30000805821B930B8F779070009789F0809136
:101B40007A0490917B048430910554F489E095E007
:101B50000E94D62380936C048A3009F0C6CDD5CD7F
:101B6000DF91CF911F910F91FF90EF90DF90CF9079
:101B7000BF90AF909F908F907F906F905F904F90AD
:101B800008958F929F92AF92BF92CF92DF92EF9281
:101B9000FF920F931F93CF93DF93F1E1EF2EF2E0CB
:101BA000FF2ECBE8D2E006EC12E0E4E8CE2EE2E035
:101BB000DE2EF70181917F010BDD882321F1F4DC1A
:101BC0004B015C01F6018081882319F46091D602F3
:101BD00001C061E070E0882777FD8095982F0E9412
:101BE000484F288139814A815B810E947B519B014A
:101BF000AC01C501B4010E94CD4DF8016083718331
:101C00008283938309C088819981AA81BB81F8016D
:101C100080839183A283B38324960C5F1F4F089423
:101C2000C11CD11CF5E1EF16F2E0FF0609F0C1CFAF
:101C300086E4CEDC8823D1F0B7DC7B018C01609395
:101C4000D7027093D8028093D9029093DA0220E0F1
:101C500030E0A9010E94A950181644F4E092F20164
:101C6000F092F3010093F4011093F501DF91CF910D
:101C70001F910F91FF90EF90DF90CF90BF90AF90AA
:101C80009F908F9008957DDF89E4A2DC882351F036
:101C90008BDC6093BA027093BB028093BC0290937A
:101CA000BD020BC080E090E0DC018093BA0290930B
:101CB000BB02A093BC02B093BD028AE489DC8823F6
:101CC00051F072DC6093BE027093BF028093C00239
:101CD0009093C102089580E090E0DC018093BE0201
:101CE0009093BF02A093C002B093C1020895CF9217
:101CF000DF92EF92FF920F931F936091C602709153
:101D0000C7028091C8029091C90220E030E0A90189
:101D10000E94A64E87FF0BC080E090E0DC0180931C
:101D2000C6029093C702A093C802B093C902609103
:101D3000CA027091CB028091CC029091CD0220E03A
:101D400030E0A9010E94A64E87FF0BC080E090E022
:101D5000DC018093CA029093CB02A093CC02B09393
:101D6000CD026091CE027091CF028091D00290910D
:101D7000D10220E030E0A9010E94A64E87FF0BC0EF
:101D800080E090E0DC018093CE029093CF02A0939C
:101D9000D002B093D1026091C6027091C7028091C7
:101DA000C8029091C90220E030E04DE453E40E9463
:101DB000A950181664F480E090E0ADE4B3E4809399
:101DC000C6029093C702A093C802B093C902609163
:101DD000CA027091CB028091CC029091CD0220E09A
:101DE00030E04DE453E40E94A950181664F480E0FA
:101DF00090E0ADE4B3E48093CA029093CB02A09349
:101E0000CC02B093CD026091CE027091CF0280914E
:101E1000D0029091D10220E030E040EF52E40E94E5
:101E2000A950181664F480E090E0A0EFB2E480932B
:101E3000CE029093CF02A093D002B093D1020E9421
:101E400002226093B2027093B3028093B402909323
:101E5000B5026091EA017091EB01882777FD8095CA
:101E6000982F0E94484F2091F2013091F301409148
:101E7000F4015091F5010E947B5120E030E040E7F1
:101E800052E40E94AD4E20E030E048EC52E40E9463
:101E9000AD4E7B018C0186EC92E06AEC72E04EEC78
:101EA00052E022ED32E0A7EACA2EA2E0DA2E0E942A
:101EB0006B2E8091C6029091C702A091C802B0918A
:101EC000C90280938B0290938C02A0938D02B093F1
:101ED0008E028091CA029091CB02A091CC02B09167
:101EE000CD0280938F0290939002A0939102B093C1
:101EF00092028091CE029091CF02A091D002B09137
:101F0000D1028093930290939402A0939502B09390
:101F100096028091D2029091D302A091D402B09106
:101F2000D5028093970290939802A0939902B09360
:101F30009A021F910F91FF90EF90DF90CF9008953C
:101F40009F92AF92BF92CF92DF92EF92FF920F9348
:101F50001F93CF93DF93982E6091BA027091BB02CA
:101F60008091BC029091BD022091BE023091BF02CF
:101F70004091C0025091C1020E94B6507B018C0179
:101F80006091EA017091EB0100D000D000D0CDB794
:101F9000DEB72196882777FD8095982F0E94484FBD
:101FA0002091F2013091F3014091F4015091F5013B
:101FB0000E947B5120E030E040E752E40E94AD4EA9
:101FC00020E030E048EC52E40E94AD4E5B016C0131
:101FD000E882F9820A831B839C828091A7028D8309
:101FE0008BE892E066EC72E04AEB52E020E001E020
:101FF000B2E0EB2E0E9498258091C6029091C70214
:10200000A091C802B091C90280938B0290938C0278
:10201000A0938D02B0938E028091CA029091CB0260
:10202000A091CC02B091CD0280938F029093900248
:10203000A0939102B09392028091CE029091CF0230
:10204000A091D002B091D102809393029093940218
:10205000A0939502B09396028091D2029091D30200
:10206000A091D402B091D5028093970290939802E8
:10207000A0939902B0939A028DB79EB706960FB6B9
:10208000F8949EBF0FBE8DBF0E9402226093B202E1
:102090007093B3028093B4029093B502DF91CF9115
:1020A0001F910F91FF90EF90DF90CF90BF90AF9076
:1020B0009F900895F8940E94FF465A985A985A980B
:1020C0005A98EBEBF0E007C09091C00095FFFCCF71
:1020D0008093C600319684918823B1F7EAE3F1E05A
:1020E00007C09091C00095FFFCCF8093C600319649
:1020F00084918823B1F78091C00085FFFCCF8AE0EE
:102100008093C600FFCFEF92FF920F931F930E9420
:1021100002222091B6023091B7024091B80250914C
:10212000B902E090B202F090B3020091B4021091B3
:10213000B5026E197F09800B910B261737074807E8
:10214000590730F4211531054105510509F0B2DF79
:102150008091EE019091EF01A091F001B091F10119
:102160000097A105B10529F10E9402222091B20237
:102170003091B3024091B4025091B502621B730BCF
:10218000840B950B2091EE013091EF014091F0010D
:102190005091F101261737074807590750F49091DD
:1021A0004A0A80914B0A981721F45A985A985A98DB
:1021B0005A980E94132E1EBA1F910F91FF90EF9014
:1021C00008952F923F924F925F926F927F928F92DB
:1021D0009F92AF92BF92CF92DF92EF92FF920F93B6
:1021E0001F93DF93CF93CDB7DEB7A2970FB6F894C6
:1021F000DEBF0FBECDBF87E4EBD9882309F496C5B7
:10220000D3D90E94154F6430710509F43CC0653084
:10221000710554F46230710531F16330710554F584
:1022200077FF19C00C94D7206A35710509F429C5C8
:102230006B35710534F46C31710511F00C94D720B5
:1022400064C06B35710509F420C56C35710511F05A
:102250000C94D7201FC58091A902882321F491DC1A
:1022600046DD0C941E218091A902882319F40BDD10
:1022700081E006C08091A902882329F404DD80E072
:102280005FDE0C941E2180E5A3D9882341F08CD910
:102290000E941A4FE62EF72E082F192F03C0EE24A6
:1022A000FF24870183E594D9882369F07DD920E054
:1022B00030E04AE754E40E947B510E941A4FE62E18
:1022C000F72E082F192F0E946B410E9402225B01FA
:1022D0006C01AE0CBF1CC01ED11E0E940222609376
:1022E000B2027093B3028093B4029093B50204C01B
:1022F0000E94044481E007DF0E9402226A157B05E8
:102300008C059D05A8F30C94D7208091F201909143
:10231000F301A091F401B091F5018093DB02909359
:10232000DC02A093DD02B093DE028091EA0190917D
:10233000EB01909389028093880284E690E0909369
:10234000EB018093EA010E9402226093B202709333
:10235000B3028093B4029093B50281E00E941C3BCB
:1023600080918B0290918C02A0918D02B0918E028F
:102370008093C6029093C702A093C802B093C9028B
:1023800080918F0290919002A0919102B09192025F
:102390008093CA029093CB02A093CC02B093CD025B
:1023A0008091930290919402A0919502B09196022F
:1023B0008093CE029093CF02A093D002B093D1022B
:1023C0008091970290919802A0919902B0919A02FF
:1023D0008093D2029093D302A093D402B093D502FB
:1023E00080E090E0DC018093F2019093F301A093F0
:1023F000F401B093F50188E5EBD8882351F489E521
:10240000E7D8882331F48AE5E3D8882311F481E002
:1024100001C080E08093F601882351F488E5D8D884
:10242000882309F4E6C089E5D3D8882309F4E1C0FC
:1024300080E090E0DC0180938B0290938C02A0936B
:102440008D02B0938E0280938F0290939002A0939E
:102450009102B09392028BE892E06FE872E043E958
:1024600052E027E932E00E948D3980E090ECA9E942
:10247000B3EC8093C6029093C702A093C802B093B6
:10248000C9028093CA029093CB02A093CC02B0936E
:10249000CD022091DA013091DB014091DC015091B5
:1024A000DD012093F2013093F3014093F401509346
:1024B000F501E090DE01F090DF010091E001109164
:1024C000E101C801B7010E94A64E87FF08C0E09253
:1024D000F201F092F3010093F4011093F501609181
:1024E000F2017091F3018091F4019091F50120E0E7
:1024F00030E040E752E40E94AD4E7B018C0186EC57
:1025000092E06AEC72E04EEC52E022ED32E0B7EA83
:10251000CB2EB2E0DB2E0E946B2E0E946B410F2E61
:10252000F0E08F2EF0E09F2EF0E0AF2EF0E0BF2E17
:10253000F02D80928B0290928C02A0928D02B0922C
:102540008E0280928F0290929002A0929102B0929D
:1025500092028BE892E06FE872E043E952E027E9EB
:1025600032E00E948D3980918B0290918C02A09173
:102570008D02B0918E028093C6029093C702A09301
:10258000C802B093C90280918F0290919002A091ED
:102590009102B09192028093CA029093CB02A093D1
:1025A000CC02B093CD026091F2017091F301809161
:1025B000F4019091F50120E030E040E752E40E9400
:1025C000AD4E7B018C0186EC92E06AEC72E04EEC41
:1025D00052E022ED32E00E946B2E8092F201909246
:1025E000F301A092F401B092F5010E946B410E94A8
:1025F000153B8091F601882331F488E50E94E80AB2
:10260000882309F4DEC00F2EF0E08F2EF0E09F2E1D
:10261000F0E0AF2EF0E0BF2EF02D80928B02909272
:102620008C02A0928D02B0928E028BE892E06FE84D
:1026300072E043E952E027E932E00E948D3980E000
:1026400090ECA9E9B3EC8093C6029093C702A093E3
:10265000C802B093C9026091DA017091DB018091E8
:10266000DC019091DD016093F2017093F30180939E
:10267000F4019093F50120E030E040E752E40E943D
:10268000AD4E7B018C0186EC92E06AEC72E04EEC80
:1026900052E022ED32E0A7EACA2EA2E0DA2E0E9432
:1026A0006B2E0E946B4180928B0290928C02A092C2
:1026B0008D02B0928E028BE892E06FE872E043E9FF
:1026C00052E027E932E00E948D3980E090E0A0EAF4
:1026D000B0E48093C6029093C702A093C802B0935F
:1026E000C9026091F2017091F3018091F40190911F
:1026F000F50120E030E040E752E40E94AD4E7B015E
:102700008C0186EC92E06AEC72E04EEC52E022ED35
:1027100032E00E946B2E0E946B4180E090E0A0E2CC
:10272000B1EC8093C6029093C702A093C802B09305
:10273000C9026091DA017091DB018091DC01909116
:10274000DD0120E030E040E05FE30E947B51262F76
:10275000372F482F592F2093F2013093F3014093E4
:10276000F4015093F50120E030E040E752E40E948C
:10277000AD4E7B018C0186EC92E06AEC72E04EEC8F
:1027800052E022ED32E00E946B2E0E946B4180925B
:102790008B0290928C02A0928D02B0928E02809257
:1027A000C6029092C702A092C802B092C90280925B
:1027B000F2019092F301A092F401B092F5010E940F
:1027C000153B8091F601882331F489E50E94E80ADF
:1027D000882309F4DEC00F2EF0E08F2EF0E09F2E4C
:1027E000F0E0AF2EF0E0BF2EF02D80928F0290929D
:1027F0009002A0929102B09292028BE892E06FE870
:1028000072E043E952E027E932E00E948D3980E02E
:1028100090ECA9E9B3EC8093CA029093CB02A09309
:10282000CC02B093CD026091DE017091DF01809106
:10283000E0019091E1016093F2017093F3018093C4
:10284000F4019093F50120E030E040E752E40E946B
:10285000AD4E7B018C0186EC92E06AEC72E04EECAE
:1028600052E022ED32E0F7EACF2EF2E0DF2E0E94B6
:102870006B2E0E946B4180928F0290929002A092E8
:102880009102B09292028BE892E06FE872E043E925
:1028900052E027E932E00E948D3980E090E0A0EA22
:1028A000B0E48093CA029093CB02A093CC02B09381
:1028B000CD026091F2017091F3018091F401909149
:1028C000F50120E030E040E752E40E94AD4E7B018C
:1028D0008C0186EC92E06AEC72E04EEC52E022ED64
:1028E00032E00E946B2E0E946B4180E090E0A0E2FB
:1028F000B1EC8093CA029093CB02A093CC02B09328
:10290000CD026091DE017091DF018091E001909134
:10291000E10120E030E040E05FE30E947B51262FA0
:10292000372F482F592F2093F2013093F301409312
:10293000F4015093F50120E030E040E752E40E94BA
:10294000AD4E7B018C0186EC92E06AEC72E04EECBD
:1029500052E022ED32E00E946B2E0E946B41809289
:102960008F0290929002A0929102B0929202809275
:10297000CA029092CB02A092CC02B092CD02809279
:10298000F2019092F301A092F401B092F5010E943D
:10299000153B8091F601882331F48AE50E94E80A0C
:1029A000882309F4DEC00F2EF0E08F2EF0E09F2E7A
:1029B000F0E0AF2EF0E0BF2EF02D809293029092C7
:1029C0009402A0929502B09296028BE892E06FE892
:1029D00072E043E952E027E932E00E948D3980E05D
:1029E00090E0A4E3B3EC8093CE029093CF02A09347
:1029F000D002B093D1026091E2017091E301809125
:102A0000E4019091E5016093F2017093F3018093EA
:102A1000F4019093F50120E030E040E752E40E9499
:102A2000AD4E7B018C0186EC92E06AEC72E04EECDC
:102A300052E022ED32E0E7EACE2EE2E0DE2E0E9406
:102A40006B2E0E946B418092930290929402A0920E
:102A50009502B09296028BE892E06FE872E043E94B
:102A600052E027E932E00E948D3980E090E0A0E852
:102A7000BFE38093CE029093CF02A093D002B09395
:102A8000D1026091F2017091F3018091F401909173
:102A9000F50120E030E040E752E40E94AD4E7B01BA
:102AA0008C0186EC92E06AEC72E04EEC52E022ED92
:102AB00032E00E946B2E0E946B4180E090E0A0E02B
:102AC000B0EC8093CE029093CF02A093D002B0934B
:102AD000D1026091E2017091E3018091E401909153
:102AE000E50120E030E040E05FE30E947B51262FCB
:102AF000372F482F592F2093F2013093F301409341
:102B0000F4015093F50120E030E040E752E40E94E8
:102B1000AD4E7B018C0186EC92E06AEC72E04EECEB
:102B200052E022ED32E00E946B2E0E946B418092B7
:102B3000930290929402A0929502B0929602809293
:102B4000CE029092CF02A092D002B092D102809297
:102B5000F2019092F301A092F401B092F5010E946B
:102B6000153B88E50E94E80A8823D9F00E94DD0A17
:102B70006115710581059105A1F00E94D40A20918B
:102B80009B0230919C0240919D0250919E020E94B6
:102B9000CD4D60938B0270938C0280938D02909345
:102BA0008E0289E50E94E80A8823D9F00E94DD0A96
:102BB0006115710581059105A1F00E94D40A20914B
:102BC0009F023091A0024091A1025091A2020E9466
:102BD000CD4D60938F0270939002809391029093F9
:102BE00092028AE50E94E80A8823D9F00E94DD0A51
:102BF0006115710581059105A1F00E94D40A20910B
:102C0000A3023091A4024091A5025091A6020E9415
:102C1000CD4D6093930270939402809395029093AC
:102C200096028BE892E06FE872E043E952E027E910
:102C300032E00E948D398091DB029091DC02A091FC
:102C4000DD02B091DE028093F2019093F301A09334
:102C5000F401B093F50180918802909189029093DC
:102C6000EB018093EA010E9402226093B20270930A
:102C7000B3028093B4029093B5020E94153B0C946A
:102C8000D7201092D6020C94D72081E08093D602F0
:102C90000C94D72085E40E94E80A882311F40E944E
:102CA0006B4141E1842E42E0942E3BE9A32E32E0B9
:102CB000B32E0BE812E0EE24F40181914F010E9443
:102CC000E80A882339F1FE2DF33061F40E94D40A1A
:102CD000F801608371838283938387E992E00E9485
:102CE0003A3A18C00E94D40AF5012081318142810C
:102CF00053810E94CD4DF801608371838283938359
:102D00008BE892E06FE872E043E952E027E932E0B5
:102D10000E948D39E39424E030E0A20EB31E0C5FD4
:102D20001F4F3E2D343041F60C94D7208DE40E9485
:102D3000E80A882311F40C942D200E94D40A0E94E2
:102D4000154F6837710509F407C7693771050CF02D
:102D50005FC06C35710509F488C56D35710564F582
:102D60006A32710509F433C16B32710574F4623152
:102D7000710509F420C56F31710509F4BDC06131D9
:102D8000710511F00C94D720B1C06335710509F4B9
:102D90000EC56435710534F46235710511F00C947B
:102DA000D72002C56435710509F405C5653571057F
:102DB00011F00C94D72043C56B36710509F4F1C4AA
:102DC0006C36710574F46936710509F4BAC16A3656
:102DD00071050CF0BFC46836710511F00C94D72052
:102DE0003BC16237710509F4DCC56337710534F402
:102DF0006D36710511F00C94D72071C263377105DF
:102E000009F4C1C56737710511F00C94D720AAC623
:102E10006C3D710509F4F8C76D3D710564F5693CB9
:102E2000710509F4FFC66A3C710574F46C387105CC
:102E300009F472C16E3B710509F4EEC3693771057F
:102E400011F00C94D7208AC66C3C710509F441C777
:102E50006D3C710534F46B3C710511F00C94D72076
:102E60001BC76D3C710509F454C76E3C710511F028
:102E70000C94D720ACC781E06F32780711F40C9422
:102E8000002091E0603379078CF4E1E06D327E0739
:102E900009F4DBC7F1E06E327F0714F00C94FC1FDD
:102EA0006D3D710511F00C94D720C0C721E0653F3E
:102EB000720711F40C94122031E0663F730744F45A
:102EC00081E06039780711F00C94D7200C940F2022
:102ED00091E0663F790711F40C941420E3E0673E1B
:102EE0007E0711F00C94D7200C9418205A9A5A9A05
:102EF0005A9A5A9A0C94D7200E9402226093DF02B9
:102F00007093E0028093E1029093E2022091E30249
:102F10003091E4024091E5025091E602621B730B8E
:102F2000840B950B28EE33E040E050E00E94735292
:102F30008DB79EB708970FB6F8949EBF0FBE8DBF92
:102F40000DB71EB70F5F1F4FCE010196EDB7FEB74D
:102F50009283818383E291E0F80193838283CA01A3
:102F6000B9012CE330E040E050E00E947352F801D8
:102F700035832483778366830E94A655E6E6F1E0D5
:102F800084912DB73EB7285F3F4F0FB6F8943EBFF0
:102F90000FBE2DBF08C09091C00095FFFCCF80935D
:102FA000C600319684918823B1F7FE01319606C0A0
:102FB0009091C00095FFFCCF8093C600819188233B
:102FC000B9F78091C00085FFFCCF0C94D42083E535
:102FD0000E94E80A882311F40C94D7200E94D40A96
:102FE0007B018C0180E50E94E80A882311F40C948F
:102FF000D720C801B7010E94154F8B0177FF02C08F
:103000000C94D7206F3F710519F014F00C94D72061
:103010000E94D40A0E94154F7B01E5E1F2E0819104
:1030200091918E159F0511F40C94D72032E0E93868
:10303000F307A9F7F7FE02C00C94D7208E2D61E0AC
:103040000E9423238E2D602F0E9444238E2DB801D1
:103050000E9498220C94D7208091A7028093E702C7
:1030600084E50E94E80A882369F10E94D40A0E943C
:103070001A4F6093E702662329F1E6E6F1E007C004
:103080009091C00095FFFCCF8093C600319684914B
:103090008823B1F7E2E3F1E006C09091C00095FF0C
:1030A000FCCF8093C60081918823B9F789E095E031
:1030B00040E050E00E9486248091C00085FFFCCF54
:1030C0000C94D42083E50E94E80A882309F10E9429
:1030D000D40A7B018C01D090E702AD2CBB240E9466
:1030E000154FDC01CB016D2D0E94F941F501EE0F6A
:1030F000FF1FE955F54F91838083F501EE0FFF1F08
:10310000EE0FFF1FE155F54FE082F182028313833A
:103110000E94FE460C94D72083E50E94E80A88238B
:1031200011F40C94D7200E94D40A0E94154FDC01A0
:10313000CB010E94AF429093AA0A8093A90A0C94F3
:10314000D7208091A7028093E70284E50E94E80AD5
:10315000882361F10E94D40A0E941A4F6093E7020B
:10316000662321F1E6E6F1E007C09091C00095FFEB
:10317000FCCF8093C600319684918823B1F7E9E4AF
:10318000F1E006C09091C00095FFFCCF8093C6008F
:1031900081918823B9F789E095E040E050E00E94F2
:1031A00086248091C00085FFFCCFFEC7E0E7F2E0F7
:1031B00007C09091C00095FFFCCF8093C600319668
:1031C00084918823B1F76091E702E62FF0E0EE0FDB
:1031D000FF1FE555F54F808191810E94FF42AB01B1
:1031E000BC0189E095E021E030E00E949525EDE604
:1031F000F2E007C09091C00095FFFCCF8093C6001D
:10320000319684918823B1F76091E702E62FF0E0D0
:10321000EE0FFF1FE955F54F808191810E94FF421B
:10322000AB01BC0189E095E021E030E00E949525EA
:10323000E9E6F2E007C09091C00095FFFCCF8093D3
:10324000C600319684918823B1F78091AD0A9091A0
:10325000AE0A0E94FE45AB01BC0189E095E021E089
:1032600030E00E949525E6E6F2E007C09091C000AC
:1032700095FFFCCF8093C600319684918823B1F7E7
:103280008091A90A9091AA0A0E94FE45AB01BC0157
:1032900089E095E021E030E00E949525E2E6F2E049
:1032A00007C09091C00095FFFCCF8093C600319677
:1032B00084918823B1F78091E70290E00E94F34166
:1032C000BC0189E095E04AE050E00E94BC24809176
:1032D000C00085FFFCCF8AE08093C600AFC7809115
:1032E000A7028093E70284E50E94E80A882361F13F
:1032F0000E94D40A0E941A4F6093E702662321F1CC
:10330000E6E6F1E007C09091C00095FFFCCF809306
:10331000C600319684918823B1F7E0E6F1E006C05B
:103320009091C00095FFFCCF8093C60081918823C7
:10333000B9F789E095E040E050E00E948624809152
:10334000C00085FFFCCF30C783E50E94E80A8823D0
:1033500009F10E94D40A7B018C01D090E702AD2CC8
:10336000BB240E94154FDC01CB016D2D0E94F94159
:10337000F501EE0FFF1FE955F54F91838083F501AD
:10338000EE0FFF1FEE0FFF1FE155F54FE082F182B8
:10339000028313830E94FE460E9402223B014C01DD
:1033A0008091E70290E0880F991FFC01E955F54FE5
:1033B000408051808555954FFC010190F081E02DB2
:1033C000F8A3EF8FEE24EA94FE2C8701EFE5F2E0FC
:1033D000249129A3EBE5F2E034913AA3E7E5F2E08A
:1033E00034905AE0252E09C189A1EFE5F2E008C02A
:1033F0009091C00095FFFCCF8093C60031968491D8
:103400008823B1F76091E702E62FF0E0EE0FFF1F8F
:10341000E555F54F808191810E94FF42AB01BC01CF
:1034200089E095E021E030E00E9495258AA1EBE556
:10343000F2E008C09091C00095FFFCCF8093C600D9
:10344000319684918823B1F76091E70289E095E095
:1034500070E04AE050E00E94BC24832DE7E5F2E0F2
:1034600008C09091C00095FFFCCF8093C6003196B4
:1034700084918823B1F717FF03C0E7E7F1E026C086
:10348000C1D79B01AC01C801B701605F784D8F4F78
:103490009F4F621B730B840B950B28EE33E040E0CB
:1034A00050E00E94735289E095E0BA01A9012AE038
:1034B00030E00E9476248091C00085FFFCCF0DC0D3
:1034C0009091C00095FFFCCF8093C6008191882326
:1034D000B9F78091C00085FFFCCF2092C60092D73B
:1034E0003B014C010E94044481E00E9483108FEF55
:1034F000E8168FEFF8068FEF08078FEF180779F5BA
:103500006091E702EF8DF8A1E415F5050CF06EC6A9
:10351000E62FF0E0EE0FFF1FE555F54F808191811A
:103520000E94FF425B016C016091E702E62FF0E030
:10353000EE0FFF1FE955F54F808191810E94FF42F8
:1035400020E030E040E85FE30E94CC4D9B01AC01FD
:10355000C601B5010E94A95087FF37C03BC017FDC7
:1035600039C06091E702E62FF0E0EE0FFF1FE5554E
:10357000F54F808191810E94FF425B016C01609157
:10358000E702E62FF0E0EE0FFF1FE955F54F8081CF
:1035900091810E94FF429B01AC01C601B5010E94CE
:1035A000CC4D0E94154F262F372F482F592F57FFEC
:1035B00007C050954095309521953F4F4F4F5F4F35
:1035C00024303105410551052CF01CD7E62EF72E8D
:1035D000082F192FFFEFEF16FFEFFF06FFEF0F0782
:1035E000FFEF1F0751F017FDE5C50CD76E197F09D6
:1035F00027E26031720708F0DDC504D76619770944
:1036000088099909693E33E0730730E0830730E0A9
:10361000930708F0E9CE66CF83E50E94E80A882385
:1036200061F00E94D40A0E94154FDC01CB010E9478
:10363000AF429093AA0A8093A90AE4D67B018C0139
:10364000E4E5F2E0D490E0E5F2E0C490ECE4F2E0EE
:10365000A490BAE09B2E71C0D5D66E197F09800B5D
:10366000910B693EE3E07E07E0E08E07E0E09E0715
:1036700008F45EC06091A702E62FF0E0EE0FFF1F96
:10368000E555F54F808191810E94FF42AB01BC015D
:103690008D2DE4E5F2E008C09091C00095FFFCCFCD
:1036A0008093C600319684918823B1F789E095E034
:1036B00022E030E00E9495258C2DE0E5F2E008C084
:1036C0009091C00095FFFCCF8093C6003196849105
:1036D0008823B1F76091A70289E095E070E04AE0A5
:1036E00050E00E94BC248A2DECE4F2E008C09091E6
:1036F000C00095FFFCCF8093C6003196849188234B
:10370000B1F78091AD0A9091AE0A0E94FE45AB01DF
:10371000BC0189E095E021E030E00E949525809190
:10372000C00085FFFCCF9092C6006CD67B018C0157
:103730000E94044481E00E9483102091A90A3091E4
:10374000AA0A8091AD0A9091AE0A821793070CF4F1
:1037500083CF39C583E50E94E80A8823F1F00E94EF
:10376000D40A20E030E0A9010E94A64E87FD0FC0D8
:103770000E94D40A20E030E04FE753E40E94A950B1
:1037800018163CF00E94D40A0E941A4F03C060E051
:1037900001C06FEF6093A8020AC58FEF8093A80263
:1037A00006C51092A80203C51092870200C581E0E9
:1037B00080938702FCC483E50E94E80A882399F07D
:1037C0000E94D40A20E030E04AE754E40E947B5192
:1037D0000E941A4F6093EE017093EF018093F00105
:1037E0009093F101E4C488E50E94E80A882309F077
:1037F000F4C489E50E94E80A882309F0EEC48AE54A
:103800000E94E80A882309F0E8C485E40E94E80AD7
:10381000882309F0E2C40E946B415A980E94D64165
:10382000C6C45A9889E50E94E80A81115A988AE527
:103830000E94E80A882309F4BAC45A98B8C483E5F8
:103840000E94E80A0E94D40A20E030E04AE754E4EB
:103850000E947B510E941A4F6093B6027093B70288
:103860008093B8029093B902A2C421E132E038A358
:103870002F8F0EE115E0EEE0EE2EE5E0FE2E7AE56C
:10388000A72E75E0B72E8824EF8DF8A18191F8A3BB
:10389000EF8F0E94E80A882309F467C0F82DF330FF
:1038A00009F05CC00E94D40A1B012C0120E030E02A
:1038B00040EA51E40E94A64E87FF4AC0F8016081A9
:1038C000718182819381A20191010E94AD4ED62E19
:1038D000C72E982E792E60915205709153058091D4
:1038E000540590915505D6012B2F3A2F492D572D70
:1038F0000E947B5160935205709353058093540549
:1039000090935505F7016081718182819381D60181
:103910002B2F3A2F492D572D0E947B51F7016083A1
:10392000718382839383F5016081718182819381A8
:103930000E94464FD6012B2F3A2F492D572D0E941A
:103940007B510E941A4FF5016083718382839383B8
:10395000F801208231824282538207C00E94D40A39
:10396000F801608371838283938383940C5F1F4F7C
:1039700024E030E0E20EF31EA20EB31E382D3430E8
:1039800009F082CF14C4E1EBF1E007C09091C000D0
:1039900095FFFCCF8093C600319684918823B1F7C0
:1039A00006C4EEEAF1E007C09091C00095FFFCCF9D
:1039B0008093C600319684918823B1F740918B02A1
:1039C00050918C0260918D0270918E0289E095E099
:1039D00022E030E00E949525EBEAF1E007C09091EB
:1039E000C00095FFFCCF8093C60031968491882358
:1039F000B1F740918F0250919002609191027091C5
:103A0000920289E095E022E030E00E949525E8EA04
:103A1000F1E007C09091C00095FFFCCF8093C600F5
:103A2000319684918823B1F740919302509194028A
:103A3000609195027091960289E095E022E030E075
:103A40000E949525E5EAF1E007C09091C00095FF3E
:103A5000FCCF8093C600319684918823B1F74091C2
:103A60009702509198026091990270919A0289E0B0
:103A700095E022E030E00E949525EBE9F1E007C0F7
:103A80009091C00095FFFCCF8093C6003196849141
:103A90008823B1F70E94C4410E94484F20911E051F
:103AA00030911F0540912005509121050E94AD4E97
:103AB000AB01BC0189E095E022E030E00E94952551
:103AC000E8E9F1E007C09091C00095FFFCCF80933A
:103AD000C600319684918823B1F781E00E94C441E9
:103AE0000E94484F209122053091230540912405E2
:103AF000509125050E94AD4EAB01BC0189E095E0D7
:103B000022E030E00E949525E5E9F1E007C09091C0
:103B1000C00095FFFCCF8093C60031968491882326
:103B2000B1F782E00E94C4410E94484F20912605CF
:103B30003091270540912805509129050E94AD4EEE
:103B4000AB01BC0189E095E022E030E0EED7809146
:103B5000C00085FFFCCF28C380E001C081E00E9447
:103B60001C3B25C3EEE8F1E007C09091C00095FF33
:103B7000FCCF8093C600319684918823B1F783B13E
:103B800080FD03C0EDE1F1E009C0E0E2F1E006C034
:103B90009091C00095FFFCCF8093C600819188234F
:103BA000B9F7E7E8F1E007C09091C00095FFFCCFBE
:103BB0008093C600319684918823B1F7199903C088
:103BC000EDE1F1E009C0E0E2F1E006C09091C00053
:103BD00095FFFCCF8093C60081918823B9F7E0E878
:103BE000F1E007C09091C00095FFFCCF8093C60024
:103BF000319684918823B1F71A9903C0EDE1F1E081
:103C000009C0E0E2F1E006C09091C00095FFFCCF52
:103C10008093C60081918823B9F78091C00085FF09
:103C2000FCCFC2C261E1E62E62E0F62E00E010E0B9
:103C3000F70181917F010E94E80A882339F10E94EF
:103C4000D40A5EE2C52E55E0D52EC00ED11E0E94CC
:103C50001A4FF60160837183828393830E94D40A92
:103C60004AE5C42E45E0D42EC00ED11EF801E25E16
:103C7000FA4F20813181428153810E947B510E9401
:103C80001A4FF60160837183828393830C5F1F4F09
:103C90000031110569F68BC201E112E03EE0E32E2E
:103CA00035E0F32EF80181918F010E94E80A882304
:103CB00039F00E94D40AF701608371838283938371
:103CC00024E030E0E20EF31E32E00531130751F735
:103CD0006EC283E50E94E80A882351F00E94D40A4C
:103CE0006093420570934305809344059093450586
:103CF00084E50E94E80A882309F459C20E94D40A84
:103D00006093460570934705809348059093490555
:103D10004EC283E50E94E80A882351F00E94D40A2B
:103D200060933E0570933F05809340059093410555
:103D300084E50E94E80A882351F00E94D40A609327
:103D4000560570935705809358059093590582E462
:103D50000E94E80A882361F00E94D40A0E941A4F48
:103D600060930A0570930B0580930C0590930D05E5
:103D700088E50E94E80A882351F00E94D40A6093E3
:103D80004A0570934B0580934C0590934D058AE549
:103D90000E94E80A882351F00E94D40A60934E05DD
:103DA00070934F05809350059093510585E40E94D0
:103DB000E80A882309F4FBC10E94D40A60935205E3
:103DC000709353058093540590935505F0C101E11C
:103DD00012E02BE9E22E22E0F22EF80181918F0110
:103DE0000E94E80A882339F00E94D40AF701608310
:103DF00071838283938324E030E0E20EF31E32E08D
:103E00000431130751F7D3C183E50E94E80A8823E0
:103E100009F4CDC10E94D40A0E94154F7093EB01A2
:103E20006093EA0181E080938A02C1C183E50E9428
:103E3000E80A882309F4BBC10E94D40A0E94154FE6
:103E40007093ED016093EC01B2C180E50E94E80A35
:103E5000882351F00E94D40A6093FC017093FD0105
:103E60008093FE019093FF0189E40E94E80A882371
:103E700081F00E94D40A25E93FEB46ED5DE30E9404
:103E80007B51609300027093010280930202909331
:103E9000030284E40E94E80A882381F00E94D40A85
:103EA00025E93FEB46ED5DE30E94AD4E60930402D1
:103EB00070930502809306029093070283E40E94A8
:103EC000E80A882351F00E94D40A60930802709394
:103ED000090280930A0290930B020E94DC41E9E7F9
:103EE000F1E006C09091C00095FFFCCF8093C60022
:103EF00081918823B9F7ECE7F1E006C09091C0000A
:103F000095FFFCCF8093C60081918823B9F740913B
:103F1000FC015091FD016091FE017091FF0189E06B
:103F200095E022E030E001D6E0E8F1E006C09091B3
:103F3000C00095FFFCCF8093C60081918823B9F71C
:103F4000609100027091010280910202909103023F
:103F500025E93FEB46ED5DE30E94AD4EAB01BC01B0
:103F600089E095E022E030E0E0D5E4E8F1E006C049
:103F70009091C00095FFFCCF8093C600819188236B
:103F8000B9F7609104027091050280910602909148
:103F9000070225E93FEB46ED5DE30E947B51AB0153
:103FA000BC0189E095E022E030E0BFD5E8E8F1E02F
:103FB00006C09091C00095FFFCCF8093C600819110
:103FC0008823B9F7609108027091090280910A0272
:103FD00090910B0225E93FEB46ED5DE30E947B519A
:103FE000AB01BC0189E095E022E030E09ED58091F4
:103FF000C00085FFFCCFD8C081E00E94563AD7C0F0
:1040000083E50E94E80A882319F00E94D40A04C0BC
:1040100060E070E086E193E40E942E47C8C00E94F1
:104020006B41C5C080E001C081E00E943108BFC083
:104030001092A9028091AE029091AF02A091B002BD
:10404000B091B1028093AA029093AB02A093AC020C
:10405000B093AD020E94260BAAC084E50E94E80A34
:10406000882309F45DC00E94D40A0E941A4F60930D
:10407000E702E6E6F1E0662369F107C09091C0002F
:1040800095FFFCCF8093C600319684918823B1F7C9
:10409000ECE8F1E006C09091C00095FFFCCF809362
:1040A000C60081918823B9F789E095E040E050E0AF
:1040B0002DD4EEE8F1E006C09091C00095FFFCCF52
:1040C0008093C60081918823B9F78091C00085FF55
:1040D000FCCF6AC01092A70207C09091C00095FF64
:1040E000FCCF8093C600319684918823B1F7EFE925
:1040F000F1E006C09091C00095FFFCCF8093C60010
:1041000081918823B9F76091A70289E095E070E07A
:104110004AE050E031D48091C00085FFFCCF44C01C
:10412000E6E6F1E007C09091C00095FFFCCF8093D8
:10413000C600319684918823B1F7EEE6F1E007C01E
:104140009091C00095FFFCCF8093C600319684917A
:104150008823B1F72091E8023091E90280E690E0EF
:10416000289FF001299FF00D389FF00D1124E65192
:10417000FD4F06C09091C00095FFFCCF8093C60014
:1041800081918823B9F7ECE6F1E007C09091C00077
:1041900095FFFCCF8093C600319684918823B1F7B8
:1041A0008091C00085FFFCCF8AE08093C6000E940A
:1041B000070B44C027D16093E3027093E40280931D
:1041C000E5029093E6021ED16093B2027093B302AF
:1041D0008093B4029093B502EACF0E946B4188E5C8
:1041E0000E94E80A882309F01CCB1CCBE62FF0E0E4
:1041F000EE0FFF1FE555F54F808191810E94FF4230
:104200005B016C016091E702E62FF0E0EE0FFF1F0B
:10421000E955F54F808191810E94FF4220E030E016
:1042200040E85FE30E94CD4D9B01AC01C601B501A2
:104230000E94A64E18160CF0C8C9CCC9A2960FB69B
:10424000F894DEBF0FBECDBFCF91DF911F910F91CC
:10425000FF90EF90DF90CF90BF90AF909F908F90A6
:104260007F906F905F904F903F902F900895809136
:104270007A0490917B048330910514F40E94510BD1
:1042800080917A0490917B040097C1F00E94E11024
:1042900080917A0490917B04019790937B048093A2
:1042A0007A048091E8029091E902019664E070E05E
:1042B0000E9460529093E9028093E8020E940444B5
:1042C00081E00E9483100C94593A0E94FF4680912D
:1042D000A9028823A1F581E08093A9028091AA0216
:1042E0009091AB02A091AC02B091AD028093AE026E
:1042F0009093AF02A093B002B093B102EBEBF0E069
:1043000007C09091C00095FFFCCF8093C600319606
:1043100084918823B1F7E2ECF0E007C09091C000EF
:1043200095FFFCCF8093C600319684918823B1F726
:104330008091C00085FFFCCF8AE08093C60008957D
:104340008091A9020895E82FF0E0ED55FB4FE4912C
:10435000E650E23060F48091B1008C7F8093B10030
:104360008091B10067707070862B8093B1000895C2
:10437000A4D00E9446097BDFFECF1F920F920FB69A
:104380000F9211242F933F938F939F93AF93BF93DB
:104390008091800490918104A0918204B091830463
:1043A00030918404232F2A592D3720F02D57019660
:1043B000A11DB11D209384048093800490938104F7
:1043C000A0938204B093830480917C0490917D0437
:1043D000A0917E04B0917F040196A11DB11D809330
:1043E0007C0490937D04A0937E04B0937F04BF91DE
:1043F000AF919F918F913F912F910F900FBE0F9092
:104400001F9018958FB7F894209180043091810403
:1044100040918204509183048FBFB901CA0108956D
:104420003FB7F89480917C0490917D04A0917E0424
:10443000B0917F0426B5A89B05C02F3F19F00196C7
:10444000A11DB11D3FBFBA2FA92F982F8827820F1A
:10445000911DA11DB11D9C01AD01220F331F441FF1
:10446000551F280F391F4A1F5B1FB901CA01089544
:10447000EF92FF920F931F93CF93DF937B018C01F9
:10448000CFDFEB010EC0CCDF6C1B7D0B83E0683E01
:10449000780738F00894E108F10801091109C851BA
:1044A000DC4FE114F1040105110569F7DF91CF91AB
:1044B0001F910F91FF90EF900895789484B58260DA
:1044C00084BD84B5816084BD85B5826085BD85B5B8
:1044D000816085BDEEE6F0E0808181608083E1E867
:1044E000F0E010828081826080838081816080839F
:1044F000E0E8F0E0808181608083E1EBF0E08081A2
:1045000084608083E0EBF0E0808181608083EAE773
:10451000F0E08081846080838081826080838081FC
:10452000816080838081806880831092C1000895BB
:104530001F93CF93DF93182FEB0161E084D0209776
:1045400009F44AC0CF3FD10509F449C0E12FF0E09A
:10455000ED55FB4FE491E330C1F0E43028F4E13055
:1045600051F0E230B1F50CC0E63019F1E73049F115
:10457000E43079F514C084B5806884BDC7BD32C00D
:1045800084B5806284BDC8BD2DC0809180008068E4
:1045900080938000D0938900C093880023C08091CD
:1045A0008000806280938000D0938B00C0938A004B
:1045B00019C08091B00080688093B000C093B300B0
:1045C00011C08091B00080628093B000C093B400AD
:1045D00009C0C038D1051CF4812F60E002C0812FD2
:1045E00061E052D0DF91CF911F910895833071F037
:1045F000843028F48130A1F0823021F514C0863057
:10460000B1F08730D1F08430E9F404C080918000AB
:104610008F7703C0809180008F7D80938000089504
:1046200084B58F7702C084B58F7D84BD0895809155
:10463000B0008F778093B00008958091B0008F7D97
:104640008093B000089590E0FC01ED57FB4F24915A
:10465000FC01ED59FB4FE491EE23A9F0F0E0EC5A98
:10466000FB4FA491B0E0662341F49FB7F8948C917E
:10467000209582238C939FBF08959FB7F8948C91C7
:10468000822B8C939FBF08950F931F93DF93CF933B
:104690000F92CDB7DEB7282F30E0F901ED55FB4F73
:1046A0008491F901ED57FB4F14912D593B4FF901BE
:1046B00004910023C9F0882319F0698397DF698189
:1046C000E02FF0E0E75AFB4FA491B0E0662331F40D
:1046D0009FB7F8948C911095812304C09FB7F894EC
:1046E0008C91812B8C939FBF0F90CF91DF911F9165
:1046F0000F9108951F920F920FB60F9211242F93CE
:104700003F934F935F936F938F939F93EF93FF9399
:104710006091C6002091050530910605C9010196FA
:104720008F77907040910705509108058417950781
:1047300041F02B573B4FF90160839093060580931E
:104740000505FF91EF919F918F916F915F914F912F
:104750003F912F910F900FBE0F901F9018959A01C7
:10476000AB0182E08093C00060E47BE48CE490E0E5
:104770000E9495522150304040405040CA01B9013A
:1047800022E030E040E050E00E9495523093C500B6
:104790002093C400E1ECF0E080818061808380811F
:1047A0008860808380818068808308958091070578
:1047B00090910805209105053091060528173907C5
:1047C00069F0FC01EB57FB4F208101968F779070C9
:1047D000909308058093070530E002C02FEF3FEF6C
:1047E000C9010895809107059091080590930605E9
:1047F0008093050508956F927F928F929F92AF925A
:10480000BF92CF92DF92EF92FF920F931F93DF93AD
:10481000CF93CDB7DEB7A0970FB6F894DEBF0FBE2B
:10482000CDBF5C01CB01BA01611571058105910510
:1048300031F4C50160E340E050E0A6D042C06E0113
:104840000894C11CD11CEE24FF248701622E77241A
:1048500088249924A40193010E947352F601619364
:104860006F010894E11CF11C011D111DB901CA0161
:10487000611571058105910569F7D801C701019797
:10488000A109B1096E010894C11CD11CC80ED91E22
:1048900013C0F60160816A3010F4605D01C0695C8C
:1048A000C50140E050E070D00894E108F10801092A
:1048B00011090894C108D108E114F104010511059A
:1048C00041F7A0960FB6F894DEBF0FBECDBFCF91D3
:1048D000DF911F910F91FF90EF90DF90CF90BF90ED
:1048E000AF909F908F907F906F9008952115310524
:1048F00039F48091C00085FFFCCF4093C600089535
:104900007ACF9A01AB0160E070E0F0CF9A01462FB8
:1049100050E060E070E0EACFEF92FF920F931F93B8
:10492000CF93DF93EC017A018B012115310539F426
:104930008091C00085FFFCCFE092C60016C02A30EF
:10494000310591F477FF0CC06DE240E050E01CD0DF
:1049500010950095F094E094E11CF11C011D111DCF
:10496000CE01B801A7012AE046DFDF91CF911F9168
:104970000F91FF90EF9008959A01FB01AF01662718
:1049800057FD6095762FC8CF9A01462F50E060E022
:1049900070E0C2CFCF93DF93EC016DE040E050E0D8
:1049A000F3DFCE016AE040E050E0EEDFDF91CF912F
:1049B0000895CF93DF93EC01A4DFCE01EBDFDF910D
:1049C000CF9108956F927F929F92AF92BF92CF92B4
:1049D000DF92EF92FF920F931F93CF93DF933C01EF
:1049E0007A018B01D22ECB01BA0120E030E0A9017F
:1049F0000E94A64E87FF09C0C3016DE240E050E06F
:104A0000C3DF17FB109517F91095CC2450E040E058
:104A100030E02FE311C0DA01F9016B2F742F8F2FD3
:104A2000922F20E030E040E251E40E94AD4E562F3C
:104A3000472F382F292FC394CD1468F3C801B7012D
:104A4000DA01F9012B2F342F4F2F5E2F0E94CD4D0D
:104A50005B01E82E192F7B2D0E941A4F062FF72E8F
:104A6000C82E992E0E94464F9B01AC016A2D7B2DCA
:104A70008E2D912F0E94CC4D5B01E82E192FC30182
:104A8000402F5F2D6C2D792D2AE030E02FDFDD20C7
:104A9000E1F1E1EBF1E006C09091C00095FFFCCFA1
:104AA0008093C60081918823B9F72FC06A2D7B2D92
:104AB0008E2D912F20E030E040E251E40E947B51A6
:104AC0008B01F82EE92E9701712F832F922F0E94D0
:104AD000154F9B01AC01EB01C301B9014AE050E065
:104AE0004BDFBE01882777FD8095982F0E94484FA5
:104AF0009B01AC01F701602F712F8F2F9E2F0E9419
:104B0000CC4D5B01E82E192FDA94DD2079F6DF9188
:104B1000CF911F910F91FF90EF90DF90CF90BF90BA
:104B2000AF909F907F906F9008954CCF0895089517
:104B30002F923F924F925F926F927F928F929F92AD
:104B4000AF92BF92CF92DF92EF92FF920F931F939B
:104B5000DF93CF93CDB7DEB7C055D0400FB6F894F2
:104B6000DEBF0FBECDBF4C017A8F698F3A012AA7F5
:104B70000EABEFAAA8AEB9AECAAEDBAE022F10E004
:104B8000000F111F000F111F9301200F311F3BABAE
:104B90002AABD9012D903D904D905C90FC01E00F27
:104BA000F11FC201B10120813181428153810E94F4
:104BB000CD4D6CAF7DAF8EAF9FAFBEA9EB2EFF2466
:104BC000EE0CFF1CEE0CFF1CF301EE0DFF1DFDAB08
:104BD000ECABA080B180C280D380F401EE0DFF1D4C
:104BE000C601B50120813181428153810E94CD4DA2
:104BF00021966FAF219722967FAF229723968FAF92
:104C0000239724969FAF2497FFA98F2F90E0880FBA
:104C1000991F880F991FF401E80FF91F2081318136
:104C2000428153812B8F3C8F4D8F5E8F498D5A8DE2
:104C3000840F951FDC016D917D918D919C912B8D41
:104C40003C8D4D8D5E8D0E94CC4D262F372F482FE9
:104C5000592F2F8F38A349A35AA3E98DFA8D3C967B
:104C60002996FFAFEEAF2997A98DBA8D1C962D918D
:104C70003D914D915C911F972EA73FA748AB59AB33
:104C8000D4011C962D913D914D915C911F972BA3C2
:104C90003CA34DA35EA3A20191015058298B3A8BEE
:104CA0004B8B5C8B1501260157FA509457F85094A2
:104CB000E98DFA8DE00FF11F60817181828193810E
:104CC000BCADADADFEADEFAD2B2F3A2F4F2F5E2F0C
:104CD0000E94CC4DB62EA72E882E692EE98DFA8D16
:104CE000EE0DFF1D60817181828193812196BFADA0
:104CF00021972296AFAD22972396FFAD2397249656
:104D0000EFAD24972B2F3A2F4F2F5E2F0E94CC4DC3
:104D1000F62E072F182FE92E69897A898B899C89AD
:104D20002F2D302F412F5E2D0E947B516D8B7E8B5E
:104D30008F8B988FC201B101D5012B2F3A2F482DAF
:104D4000562D0E947B519B01AC016D897E898F8914
:104D5000988D0E94CC4D6D8B7E8B8F8B988F69893F
:104D60007A898B899C89D5012B2F3A2F482D562D76
:104D70000E947B515B016C01C201B1012F2D302FCC
:104D8000412F5E2D0E947B519B01AC01C601B501F4
:104D90000E94CD4D9B01AC016D897E898F89988DD4
:104DA0000E94404E162FE72E082FF92E20E030E00B
:104DB000A9010E94A64E87FF0EC0612F7E2D802F75
:104DC0009F2D2BED3FE049EC50E40E94CD4D162F76
:104DD000E72E082FF92EAA968FADAA97882371F097
:104DE000612F7E2D802F9F2D2BED3FE049EC50E46D
:104DF0000E94CC4D162FE72E082FF92E612F7E2D05
:104E0000802F9F2DA9962CAD3DAD4EAD5FADA997DE
:104E10000E947B512F8D38A149A15AA15F770E9432
:104E2000B6505B016C012FE632E143E85AE30E9481
:104E3000A64E87FDA4C2C601B5010E94834F0E9401
:104E40001A4F7DA76CA76115710521F481E090E0F0
:104E50009DA78CA7ACA5BDA5BD0180E090E00E94F8
:104E6000464F5B016C01612F7E2D802F9F2DA60187
:104E700095010E94AD4E6D8B7FA388A799A76F8D7A
:104E800078A189A19AA1A60195010E94AD4E2A960A
:104E90006FAF2A972B967FAF2B972C968FAF2C97BF
:104EA0002D969FAF2D976EA57FA588A999A92BA1B7
:104EB0003CA14DA15EA10E94CC4DA60195010E948E
:104EC000AD4E2E966FAF2E972F967FAF2F97609691
:104ED0008FAF609761969FAF61975D894FA138A5AD
:104EE00029A5652F742F832F922F20E030E040E01A
:104EF0005FE30E947B51BD89AFA1F8A5E9A52B2FE7
:104F00003A2F4F2F5E2F0E947B519B01AC0160E036
:104F100070E080E89FE30E94CC4D6EA725967FAF9E
:104F2000259726968FAF269727969FAF2797BFA9DD
:104F3000EB2FF0E0EE0FFF1FEE0FFF1FCE010196EB
:104F4000E80FF91F2B8D3C8D4D8D5E8D20833183B5
:104F5000428353832BA13CA14DA15EA12D873E87A7
:104F60004F87588BBB2441E050E05CA34BA3BAA50C
:104F7000AB2FB0E0AA0FBB1FAA0FBB1F9C012A0FCB
:104F80003B1F3C8F2B8F5EA9452F50E0440F551FD0
:104F9000440F551F81E090E08C0F9D1F840F951FDB
:104FA00098A38F8FFBA7EAA7CAC19B2D99310CF05C
:104FB00068C069897A898B899C89BD89AFA1F8A568
:104FC000E9A52B2F3A2F4F2F5E2F0E947B517B019B
:104FD0008C01C201B101BEA52596AFAD25972696DD
:104FE000FFAD26972796EFAD27972B2F3A2F4F2F00
:104FF0005E2F0E947B519B01AC01C801B7010E944A
:10500000CD4DD62EA72E882E692E69897A898B8957
:105010009C89BEA52596AFAD25972696FFAD269710
:105020002796EFAD27972B2F3A2F4F2F5E2F0E94F9
:105030007B51162F072FF82EE92EC201B101BD8931
:10504000AFA1F8A5E9A52B2F3A2F4F2F5E2F0E9475
:105050007B519B01AC01D801F7016B2F7A2F8F2F69
:105060009E2F0E94CC4D262F372F482F592F298B4A
:105070003A8B4B8B5C8BB3942D2C3A2C482C562CB2
:105080006AC0ABA1BCA1BD0180E090E00E94464F88
:10509000BD89AFA1F8A5E9A52B2F3A2F4F2F5E2F81
:1050A0000E947B517B018C017F2D912F0E94AA4E83
:1050B0001B012C016E2D7F2D802F912F0E94DE5120
:1050C0005B016C01EAA9FBA9E080F18002811381F8
:1050D00017FB109517F91095ACA9BDA96D907D909F
:1050E0008D909C90C801B701A20191010E947B5153
:1050F000698B7A8B8B8B9C8BC401B301A6019501C4
:105100000E947B519B01AC0169897A898B899C89BA
:105110000E94CD4D262F372F482F592F298B3A8BA0
:105120004B8B5C8BC801B701A60195010E947B5196
:105130007B018C01C401B301A20191010E947B514A
:105140009B01AC01C801B7010E94CC4D262E372E21
:10515000482E592EBB245CAD4DAD3EAD2FAD652F15
:10516000742F832F922F29893A894B895C890E9459
:10517000CD4DEB8DFC8D608371838283938321966B
:105180005FAD219722964FAD229723963FAD23978F
:1051900024962FAD2497652F742F832F922FA20171
:1051A00091010E94CD4DAF8DB8A16D937D938D93EC
:1051B0009C931397EAA5FBA56081718182819381FD
:1051C0002A96BFAD2A972B96AFAD2B972C96FFADA5
:1051D0002C972D96EFAD2D972B2F3A2F4F2F5E2F1B
:1051E0000E94CD4DAAA5BBA56D937D938D939C93F5
:1051F00013976D857E858F8598892E96BFAD2E97E6
:105200002F96AFAD2F976096FFAD60976196EFAD8B
:1052100061972B2F3A2F4F2F5E2F0E94CD4D6D8718
:105220007E878F87988B69817A818B819C8120E032
:1052300030E0A9010E94A64E87FF07C080E090E001
:10524000DC0189839A83AB83BC836D817E818F81EE
:10525000988520E030E0A9010E94A64E87FF07C094
:1052600080E090E0DC018D839E83AF83B887698501
:105270007A858B859C8520E030E0A9010E94A64EAE
:1052800087FF07C080E090E0DC0189879A87AB87C1
:10529000BC8769817A818B819C8120E030E04DE47C
:1052A00053E40E94A950181644F480E090E0ADE465
:1052B000B3E489839A83AB83BC836D817E818F81C4
:1052C000988520E030E04DE453E40E94A950181680
:1052D00044F480E090E0ADE4B3E48D839E83AF833B
:1052E000B88769857A858B859C8520E030E040EF22
:1052F00052E40E94A950181644F480E090E0A0EF18
:10530000B2E489879A87AB87BC87CE010196BE013C
:105310006B5F7F4FAE01475F5F4F9E01235F3F4F43
:10532000E8ACF9AC0AAD1BADFAE6CF2ED12CCC0E11
:10533000DD1ED1D4EBA1FCA13196FCA3EBA32BA1E4
:105340003CA14CA55DA52417350708F42ECE698D28
:105350007A8D6C5F7F4F498D5A8D485F5F4F898D85
:105360009A8D29962EAD3FAD2997E8ACF9AC0AADE0
:105370001BADEAE6CE2ED12CCC0EDD1EACD4C05B2C
:10538000DF4F0FB6F894DEBF0FBECDBFCF91DF91D8
:105390001F910F91FF90EF90DF90CF90BF90AF9053
:1053A0009F908F907F906F905F904F903F902F9045
:1053B00008958F5F803109F480E008952F923F9225
:1053C0004F925F926F927F928F929F92AF92BF9215
:1053D000CF92DF92EF92FF920F931F93DF93CF93C1
:1053E000CDB7DEB76A970FB6F894DEBF0FBECDBF5C
:1053F0009A8F898F3A014B0178018901DC01D89697
:105400006D917D918D919C91DB970E94464F5B0140
:105410006C01A40193010E947B510E94934E0E9453
:105420001A4F262F372F482F592F2D873E874F870A
:10543000588BC601B501A80197010E947B510E94BB
:10544000934E0E941A4F9B01AC01298B3A8B4B8BD8
:105450005C8B8D859E85AF85B88988379105A105C0
:10546000B10540F488E790E0A0E0B0E08D879E872A
:10547000AF87B88B283731054105510540F428E73F
:1054800030E040E050E0298B3A8B4B8B5C8BE98D10
:10549000FA8DEC5BFF4F6080718082809380A98DD4
:1054A000BA8DDC966D917D918D919C91DF970E94D4
:1054B000464F6D837E838F839887C401B3010E941A
:1054C000484F1B012C0120E030E0A9010E94A64EAC
:1054D000882329F1C601B501A60195010E947B51DF
:1054E0007B018C016D817E818F8198859B01AC0150
:1054F0000E947B519B01AC01C801B7010E94CC4DB9
:105500007B018C01C201B101A20191010E94CD4D2C
:105510009B01AC01C801B7010E94AD4E04C060E020
:1055200070E080E090E00E94934E0E94154F6983E6
:105530007A838B839C83E980FA800B811C81E98DBF
:10554000FA8DE05CFF4F60817181828193810E94BE
:10555000464F69877A878B879C8766277727CB0199
:1055600066197709880999090E94484F3B014C0147
:1055700020E030E0A9010E94A64E882349F1698508
:105580007A858B859C859B01AC010E947B516D8B3C
:105590007E8B8F8B988FC601B501A60195010E9465
:1055A0007B519B01AC016D897E898F89988D0E940A
:1055B000CC4D5B016C01C401B301A40193010E94B5
:1055C000CD4D9B01AC01C601B5010E94AD4E04C09A
:1055D00060E070E080E090E00E94834FE98DFA8DFA
:1055E000A088B188C288D3883501460129813A81D3
:1055F0004B815C81621A730A840A950A0E94154FD6
:10560000A4019301261B370B480B590BDA01C90182
:1056100057FF68C0C201B10120E030E0A9010E943B
:10562000A64E882309F443C0C201B101A201910131
:105630000E94CD4D7B018C01C601B5010E94464FF1
:105640009B01AC01C801B7010E947B517B018C0119
:105650006D817E818F8198859B01AC010E947B5179
:105660009B01AC01C801B7010E94CC4D7B018C01AC
:1056700069857A858B859C859B01AC010E947B5155
:105680009B01AC01C801B7010E94CD4D7B018C018B
:10569000C201B10120E030E040E850E40E947B51BB
:1056A0009B01AC01C801B7010E94AD4E04C060E08F
:1056B00070E080E090E00E94934E0E94154FE62E2D
:1056C000F72E082F192F17FF03C0EE24FF248701A0
:1056D000EA14FB040C051D0510F08601750180E03D
:1056E00090E0DC012FB7F894E98DFA8DE45BFF4F71
:1056F0003081332311F5E98DFA8DE48AF58A068B22
:10570000178BE80EF91E0A1F1B1FE08EF18E028F09
:10571000138F8D859E85AF85B88984AF95AFA6AF71
:10572000B7AFAF01405C5F4F89899A89AB89BC896B
:10573000FA0180839183A283B3832FBF6A960FB649
:10574000F894DEBF0FBECDBFCF91DF911F910F91B7
:10575000FF90EF90DF90CF90BF90AF909F908F9091
:105760007F906F905F904F903F902F9008959F9201
:10577000AF92BF92CF92DF92EF92FF920F931F935F
:10578000CF93DF93EB017A01209709F46EC04115A6
:10579000510509F46AC01AA5BBA4ACA49DA46EA1CE
:1057A0007FA188A599A5212F3B2D4A2D592D0E9417
:1057B000A64E882309F459C08FA9882309F047C051
:1057C000F701C6A0D7A0E0A4F1A4612F7B2D8A2DFC
:1057D000992DA70196010E94A9501816C4F5C7017A
:1057E000B601A70196010E947B516B017C012AA999
:1057F0003BA94CA95DA95058CA01B9010E94CD4DE1
:105800002EA53FA548A959A90E947B519B01AC0137
:10581000C701B6010E94CC4D0E94E851C62E072F49
:10582000F82EE92E612F7B2D8A2D992DF7012C2D35
:10583000302F4F2F5E2F0E94A64E87FF04C0C12E2F
:105840000B2DFA2CE92C5C2D402F970104C0512F11
:105850004B2D3A2D292D852F942FA32FB22F8EA3B8
:105860009FA3A8A7B9A781E08EABDF91CF911F912D
:105870000F91FF90EF90DF90CF90BF90AF909F90EF
:105880000895CF92DF92EF92FF920F931F93DF93D1
:10589000CF930F92CDB7DEB780914A0A80914A0A22
:1058A00020914B0A90E04096821B91098F70907076
:1058B0008430910544F120914A0A23502F7040E032
:1058C00050E000E010E08DE4E82EF12C18C0222317
:1058D00009F420E12150822F90E08E9D60018F9D80
:1058E000D00C9E9DD00C11248AE795E0C80ED91EDD
:1058F000C601B80129833BDFA80186012981809177
:105900004B0A281721F70F90CF91DF911F910F912C
:10591000FF90EF90DF90CF9008958F929F92AF927B
:10592000BF92CF92DF92EF92FF920F931F93CF938C
:10593000DF93EC016B01009709F465C08FA9882300
:1059400009F061C0EEA0FFA008A519A5FB01B6A053
:10595000A7A090A481A4C801B701D501F4012B2F01
:105960003A2F4F2F5E2F0E94A64E87FF4CC0C801D2
:10597000B701A80197010E947B517B018C012AA9E4
:105980003BA94CA95DA95058CA01B9010E94CD4D4F
:105990002EA53FA548A959A90E947B519B01AC01A6
:1059A000C801B7010E94CC4D0E94E8518B017C01D7
:1059B000A5019401652F742F832F922F202F312F53
:1059C0004E2D5F2D0E94A64E87FF04C00B2D1A2D71
:1059D000E92CF82CA5019401652F7A2D832F982DA1
:1059E000202F312F4E2D5F2D0E94A64E882359F077
:1059F000802F912FAE2DBF2DF60186A397A3A0A7D0
:105A0000B1A781E086ABDF91CF911F910F91FF90FD
:105A1000EF90DF90CF90BF90AF909F908F900895C0
:105A2000DF92EF92FF920F931F93CF93DF93D0906B
:105A30004B0A00E010E080E090E02DE4E22EF12C33
:105A400013C02D2D30E02E9DE0012F9DD00D3E9DE9
:105A5000D00D1124C658DA4FB801AE015EDF8D2D8E
:105A6000A8DCD82EC8018E0120914A0AD21649F727
:105A7000B80140E050E051DFDF91CF911F910F91CD
:105A8000FF90EF90DF9008952F923F924F925F9298
:105A90006F927F928F929F92AF92BF92CF92DF923E
:105AA000EF92FF920F931F93CF93DF93F0904B0AE7
:105AB000C0E0D0E03DE4632E712C3EC0069D600145
:105AC000079DD00C169DD00C11248AE795E0C80ED6
:105AD000D91E209769F18EA9882321F4F60186A9A1
:105AE000882331F18AA09BA0ACA0BDA06EA17FA1AC
:105AF00088A599A5A50194010E94AD4E1B012C011A
:105B0000069DF001079DF00D169DF00D1124E6583D
:105B1000FA4F66A177A180A591A5A50194010E94E5
:105B2000AD4E8B019C01CE01B201A10147DC1EAA42
:105B30008F2D3FDCF82EE6010F2D112707FD109564
:105B400080914A0A90E00817190709F0B7CF20970B
:105B5000E9F0CAA0DBA0ECA0FDA06EA17FA188A502
:105B600099A5A70196010E94AD4E4B015C016DEC19
:105B70007CEC8CE49DE3A70196010E94AD4E8B0165
:105B80009C01CE01B501A40119DC1EAADF91CF91C1
:105B90001F910F91FF90EF90DF90CF90BF90AF904B
:105BA0009F908F907F906F905F904F903F902F903D
:105BB000089567DE35DF68CF10924A0A10924B0ACB
:105BC00080E1EAE6F5E0DF011D928A95E9F780E0E1
:105BD00090E0DC018093510A9093520AA093530AFB
:105BE000B093540A8093550A9093560AA093570A8B
:105BF000B093580A8093590A90935A0AA0935B0A6B
:105C0000B0935C0A80935D0A90935E0AA0935F0A4A
:105C1000B093600A80934D0A90934E0AA0934F0A66
:105C2000B093500A08951F9390914B0A80914A0AAD
:105C3000981779F140914B0A242F30E08DE490E0E1
:105C4000289FF001299FF00D389FF00D1124EE538D
:105C5000FA4F108150E02DE430E016C0842F90E020
:105C6000829FF001839FF00D929FF00D1124EE535F
:105C7000FA4F80819181A281B3810097A105B1057E
:105C800009F05F5F4F5F4F7080914A0A481731F704
:105C90000AC06091A802662321F08EE070E00E94A5
:105CA000982210E050E08091A802882339F455230F
:105CB00029F48EE060E070E00E9498228091A802B2
:105CC000882339F0112329F08EE0612F70E00E94C3
:105CD00098221F9108952F923F924F925F926F9258
:105CE0007F928F929F92AF92BF92CF92DF92EF926C
:105CF000FF920F931F93DF93CF93CDB7DEB7CF54AF
:105D0000D0400FB6F894DEBF0FBECDBF5C011B01C3
:105D10003A013AA329A34E2C8F2C902EF12ED8AE07
:105D2000CFAA80914A0A45DB2C968FAF2C97082F7B
:105D3000112707FD109505C00E94044481E00E94D0
:105D4000831080914B0A90E080179107A9F3D50149
:105D50006D917D918D919C9120911E0530911F0533
:105D600040912005509121050E947B510E944B518A
:105D70006BAF7CAF8DAF9EAFF1016081718182818D
:105D80009381209122053091230540912405509163
:105D900025050E947B510E944B516FAF21967FAF2A
:105DA000219722968FAF229723969FAF2397D301F7
:105DB0006D917D918D919C912091260530912705C3
:105DC00040912805509129050E947B510E944B511A
:105DD00024966FAF249725967FAF259726968FAF91
:105DE000269727969FAF2797E9A1FAA16081718135
:105DF0008281938120912A0530912B0540912C05B9
:105E000050912D050E947B510E944B516BAB7CAB96
:105E10008DAB9EAB8091760590917705A09178052A
:105E2000B0917905ABA8BCA8CDA8DEA8A816B90684
:105E3000CA06DB0609F445C06091A702E62FF0E030
:105E4000EE0FFF1FE555F54F808191810E94FF42C3
:105E500020E030E046E153E40E94A64E87FF31C0C7
:105E600080914C0A882369F52BA93CA94DA95EA90C
:105E70002093760530937705409378055093790504
:105E8000E3ECF4E007C09091C00095FFFCCF809355
:105E9000C600319684918823B1F7E7EEF4E007C09D
:105EA0009091C00095FFFCCF8093C60031968491FD
:105EB0008823B1F78091C00085FFFCCF8AE08093F2
:105EC000C6008091760590917705A0917805B091F4
:105ED0007905ABA8BCA8CDA8DEA8A81AB90ACA0A39
:105EE000DB0AC601B501D7FE07C090958095709575
:105EF00061957F4F8F4F9F4F0E94484F5B016C0110
:105F000060912A0570912B0580912C0590912D05AB
:105F100020E030E04DEC53E40E947B519B01AC014A
:105F2000C601B5010E94A95018166CF52BA93CA911
:105F30004DA95EA9209376053093770540937805A7
:105F400050937905E3ECF4E007C09091C00095FF11
:105F5000FCCF8093C600319684918823B1F7E9EC99
:105F6000F4E007C09091C00095FFFCCF8093C6007D
:105F7000319684918823B1F78091C00085FFFCCFD2
:105F80008AE08093C60080914A0A482F50E05AA3C5
:105F900049A38DE490E0489FF001499FF00D589F80
:105FA000F00D1124E658FA4FDF01A45BBF4F1C929D
:105FB00060916A0570916B0580916C0590916D05FB
:105FC0006BA37CA38DA39EA38BAD9CADADADBEADED
:105FD000ABA0BCA0CDA0DEA08A199B09AC09BD096D
:105FE000B7FF07C0B095A095909581959F4FAF4F93
:105FF000BF4F80839183A283B38320916E0530913C
:106000006F0540917005509171052BA73CA74DA7D6
:106010005EA78DE490E049A15AA1489FF001499FF5
:10602000F00D589FF00D1124E658FA4F23968CADD1
:106030009DADAEADBFAD2397ABA4BCA4CDA4DEA4F3
:106040008A199B09AC09BD09B7FF07C0B095A09597
:10605000909581959F4FAF4FBF4F84839583A683C3
:10606000B78320917205309173054091740550916A
:1060700075052FA738AB49AB5AAB8DE490E049A129
:106080005AA1489FF001499FF00D589FF00D11242F
:10609000E658FA4F27968CAD9DADAEADBFAD2797B4
:1060A000AFA4B8A8C9A8DAA88A199B09AC09BD0988
:1060B000B7FF07C0B095A095909581959F4FAF4FC2
:1060C000BF4F80879187A287B38720917605309153
:1060D000770540917805509179052FA338A749A7F6
:1060E0005AA72091EC013091ED016BA97CA98DA9F3
:1060F0009EA9AFA0B8A4C9A4DAA46A197B098C0927
:106100009D0997FF07C090958095709561957F4F89
:106110008F4F9F4F442737FD4095542F0E94415287
:1061200024E630E040E050E00E9495528DE490E09B
:10613000C9A0DAA0C89EF001C99EF00DD89EF00D4E
:106140001124E658FA4F2487358746875787008100
:10615000118172816381A480B580C680D7808085DB
:106160009185A285B3858A159B05AC05BD0514F400
:10617000D601C50182179307A407B50714F4DA0105
:10618000C901FB01202F312F4F2F562F2817390718
:106190004A075B0714F49C01AD018DE490E069A10E
:1061A0007AA1689FF001699FF00D789FF00D11248E
:1061B000E658FA4F208B318B428B538B26303105BA
:1061C0004105510510F40C9473399F01285B3F4F32
:1061D0008091A802482F50E060E070E0D9014D9313
:1061E0005D936D937C93139710A2ABACBCACCDAC1C
:1061F000DEAC2BA13CA14DA15EA1A216B306C40644
:10620000D50614F481E080A323964CAD5DAD6EAD50
:106210007FAD23978BA59CA5ADA5BEA548175907B3
:106220006A077B0784F48DE490E0A9A1BAA1A89F36
:10623000F001A99FF00DB89FF00D1124E658FA4F18
:1062400080A1826080A32796ACACBDACCEACDFACA5
:1062500027972FA538A949A95AA9A216B306C4069B
:10626000D50684F48DE490E049A15AA1489FF0013D
:10627000499FF00D589FF00D1124E658FA4F80A168
:10628000846080A36BA97CA98DA99EA9AFA0B8A4A6
:10629000C9A4DAA46A157B058C059D0584F48DE4F8
:1062A00090E0C9A0DAA0C89EF001C99EF00DD89E6A
:1062B000F00D1124E658FA4F80A1886080A38DE488
:1062C00090E029A13AA1289FF001299FF00D389F65
:1062D000F00D1124E658FA4FAFA9B8AD8C9181A307
:1062E00080819181A281B3810097A105B10509F058
:1062F0005A9A8DE490E0A9A0BAA0A89EF001A99EA8
:10630000F00DB89EF00D1124E658FA4F8481958166
:10631000A681B7810097A105B10509F05A9A8DE4CD
:1063200090E0C9A0DAA0C89EF001C99EF00DD89EE9
:10633000F00D1124E658FA4F80859185A285B3852A
:106340000097A105B10509F05A9A8DE490E029A1C2
:106350003AA1289FF001299FF00D389FF00D1124DC
:10636000E658FA4F84859585A685B7850097A105DF
:10637000B10509F05A9A8DE490E049A15AA1489FCD
:10638000F001499FF00D589FF00D1124E658FA4F87
:1063900084859585A685B7850097A105B10549F443
:1063A000E090560500915705109158053090590519
:1063B00008C0E0903E0500913F05109140053090E7
:1063C0004105642D782D892D9F2D2E2D302F412FA5
:1063D000532D0E94A64E87FD03C0E42C84013F2C60
:1063E00080916A0590916B05A0916C05B0916D0547
:1063F000ABACBCACCDACDEACA81AB90ACA0ADB0A9D
:10640000C601B5010E94484F20911E0530911F051D
:1064100040912005509121050E94AD4EF62E772E19
:10642000682E9BA3292F862F972DA62DB22F898307
:106430009A83AB83BC8380916E0590916F05A09188
:106440007005B091710523962CAD3DAD4EAD5FAD9D
:106450002397281B390B4A0B5B0BCA01B9010E9419
:10646000484F2091220530912305409124055091F9
:1064700025050E94AD4E562E472E8BA79FA7A20141
:10648000382F292F852F942FA32FB22F8D839E83F2
:10649000AF83B8878091720590917305A0917405C0
:1064A000B09175052796ACACBDACCEACDFAC2797F0
:1064B000A81AB90ACA0ADB0AC601B5010E94484FE8
:1064C00020912605309127054091280550912905F6
:1064D0000E94AD4E262E7FA38FAB28969FAF2897A4
:1064E000472F382F292F862F942FA32FB22F89873C
:1064F0009A87AB87BC878090EC019090ED018091EA
:10650000760590917705A0917805B09179052BA932
:106510003CA94DA95EA9281B390B4A0B5B0BCA018C
:10652000B9010E94484F20912A0530912B054091D6
:106530002C0550912D050E94AD4E5B016C01B401FC
:10654000882777FD8095982F0E94484F9B01AC01CA
:10655000C601B5010E947B5120E030E048EC52E4D6
:106560000E94AD4E262F372F482F592F6D877E87DB
:106570008F87988B8DE490E069A17AA1689FF001E4
:10658000699FF00D789FF00D1124E658FA4F808135
:106590009181A281B38186309105A105B105C4F432
:1065A00084819581A681B78186309105A105B105C9
:1065B0007CF480859185A285B38586309105A105FF
:1065C000B10534F45F7726A737A740AB51AB42C083
:1065D0002BA16F2D772D862D922F0E9426525B01C5
:1065E0006C01A2013BA52FA5652F742D832F922F3F
:1065F0000E9426522B013C014FA13FA928962FADA6
:106600002897622D742F832F922F0E9426526BA3FE
:106610007CA38DA39EA3C601B501A30192010E9494
:10662000CD4D2BA13CA14DA15EA10E94CD4D0E945C
:10663000E8512DE430E0A9A1BAA1A29FF001A39FE7
:10664000F00DB29FF00D1124E658FA4F66A777A718
:1066500080AB91AB8DE490E0A9A0BAA0A89EF00118
:10666000A99EF00DB89EF00D1124E658FA4F26A50C
:1066700037A540A951A92FA338A749A75AA760E079
:1066800070E080E89FE30E94AD4E9B01AC016E2D4F
:10669000702F812F932D0E947B51362E272E8BA792
:1066A0009FA790914A0A80914B0A492F50E0405F82
:1066B0005F4F481B51094F7050705CA34BA360E0C3
:1066C00074E284E799E4D101FBA5EFA52B2F3A2FC3
:1066D0004F2F5E2F0E94AD4E0E944B51962E872E5B
:1066E000682E492E6BA17CA1623071050CF44AC062
:1066F0005B01CC24B7FCC094DC2CC601B5010E9420
:10670000484F20E030E040E051E40E94A64E87FF71
:1067100039C0E92CF82C062D142D60910A057091D2
:106720000B0580910C0590910D05E616F7060807FC
:10673000190740F56E197F09800B910B660F771FC3
:10674000881F991FA60195010E947352CA01B901C1
:106750000E94464F0E944B519B01AC01CA01B901F6
:106760006E0D7F1D801F911F0E94464F9B01AC0143
:1067700060E074E284E799E40E94AD4E362E272E45
:106780008BA79FA78DE490E0A9A1BAA1A89F800143
:10679000A99F100DB89F100D112406581A4F6FA114
:1067A00078A589A59AA5D101FBA5EFA52B2F322DA0
:1067B0004F2F5E2F0E947B51F80162A373A384A325
:1067C00095A360897189828993890E94464FD1017E
:1067D000FBA5EFA52B2F322D4F2F5E2F0E947B5153
:1067E0000E94934E0E941A4FD801D8966D937D93C4
:1067F0008D939C93DB97FE013196F8A7EFA38E0152
:106800000F5E1F4F2EE035E029963FAF2EAF299740
:1068100018AF0FABEE24FF24B0E8DB2EAFE3CA2E97
:10682000AFA1B8A56D917D918D919D91B8A7AFA3B2
:10683000D101FBA5EFA52B2F322D4F2F5E2F0E94EC
:106840007B519B01AC01EFA9F8AD219331934193AA
:106850005193F8AFEFAB29013A01E89477F8299604
:10686000AEADBFAD29978D909D90AD90BD9029960E
:10687000BFAFAEAF2997C301B201A50194010E9439
:10688000A9501816E4F4C501B401A30192010E94B5
:10689000AD4EB62EA72E982E892E96016E2D7F2DE9
:1068A000832F9C2DD501F4012B2F3A2F4F2F5E2FD4
:1068B0000E94A64E87FD03C0EB2CFA2C6401EFA1C9
:1068C000F8A5E017F10709F0ABCF96016E2D7F2DEB
:1068D000832F9C2D20E030E040E85FE30E94A64E2D
:1068E00087FF50C0F1E2AF2EB12CAC0EBD1ED80117
:1068F0006D917D918D919C91F6012E2D3F2D4F2F05
:106900005C2D0E947B51F801619371938193919367
:106910008F01EA15FB0559F78DE490E0A9A0BAA014
:10692000A89E8001A99E100DB89E100D1124065836
:106930001A4FD80192966D917D918D919C9195976A
:10694000F6012E2D3F2D4F2F5C2D0E947B51F8011B
:1069500062A373A384A395A360AD71AD82AD93AD23
:106960000E94464FF6012E2D3F2D4F2F5C2D0E9489
:106970007B510E941A4FD801D8966D937D938D93C9
:106980009C93DB978DE490E0E9A1FAA1E89F800158
:10699000E99F100DF89F100D112406581A4FD801C9
:1069A00050966D917D918D919C9153970E94464F89
:1069B000F80126A537A540A951A90E94AD4E762E13
:1069C000672E382E292EF80180819181A281B38112
:1069D0000097A105B10569F584819581A681B781EC
:1069E0000097A105B10529F580859185A285B3851C
:1069F0000097A105B105E9F4A3019101652F742F5A
:106A0000832F922F209146053091470540914805EC
:106A1000509149050E947B510E94934E0C5B1F4F81
:106A20000E941A4FD8016D937D938D939C93139779
:106A300065C1A3019101652F762D832F922D2091A1
:106A400042053091430540914405509145050E940F
:106A50007B510E94934E0E941A4F2DE430E0E9A131
:106A6000FAA1E29F8001E39F100DF29F100D112407
:106A700006581A4FE4E44E2E512C400E511ED201FE
:106A80006D937D938D939C93139780905A0590906E
:106A90005B05A0905C05B0905D050E94464F6B01C0
:106AA0007C01F80160817181828193810E94484F4D
:106AB0009B01AC01C701B6010E947B516B017C01B7
:106AC000D80150966D917D918D919C9153970E9424
:106AD000464F9B01AC01C701B6010E94AD4E7B0140
:106AE0008C01C501B4010E94464F9B01AC01C80155
:106AF000B7010E94A95018162CF4F20180829182ED
:106B0000A282B38280905E0590905F05A0906005A0
:106B1000B09061058DE490E0C9A0DAA0C89E800124
:106B2000C99E100DD89E100D112406581A4F64E40A
:106B3000462E512C400E511ED2016D917D918D91AA
:106B40009C910E94464F6B017C01F8016481758124
:106B5000868197810E94484F9B01AC01C701B60115
:106B60000E947B516B017C01D80150966D917D9103
:106B70008D919C9153970E94464F9B01AC01C70198
:106B8000B6010E94AD4E7B018C01C501B4010E948B
:106B9000464F9B01AC01C801B7010E94A9501816CD
:106BA0002CF4F20180829182A282B38280906605E9
:106BB00090906705A0906805B09069058DE490E01D
:106BC000C9A0DAA0C89E8001C99E100DD89E100DE4
:106BD000112406581A4F54E4452E512C400E511ED4
:106BE000D2016D917D918D919C910E94464F6B01D8
:106BF0007C01F80164857585868597850E94484FDC
:106C00009B01AC01C701B6010E947B516B017C0165
:106C1000D80150966D917D918D919C9153970E94D2
:106C2000464F9B01AC01C701B6010E94AD4E7B01EE
:106C30008C01C501B4010E94464F9B01AC01C80103
:106C4000B7010E94A95018162CF4F201808291829B
:106C5000A282B3828090620590906305A090640543
:106C6000B09065058DE490E0C9A0DAA0C89E8001CF
:106C7000C99E100DD89E100D112406581A4F44E4D9
:106C8000442E512C400E511ED2016D917D918D915B
:106C90009C910E94464F6B017C01F80160857185D3
:106CA000828593850E94484F9B01AC01C701B601C4
:106CB0000E947B516B017C01D80150966D917D91B2
:106CC0008D919C9153970E94464F9B01AC01C70147
:106CD000B6010E94AD4E7B018C01C501B4010E943A
:106CE000464F9B01AC01C801B7010E94A95018167C
:106CF0002CF4F20180829182A282B3828DE490E032
:106D0000A9A0BAA0A89E8001A99E100DB89E100D42
:106D1000112406581A4FF801EC5BFF4F6081718116
:106D2000828193810E94464F6B017C01D301F10166
:106D30002B2F362D4F2F522D0E94AD4ED801D296BB
:106D40006D937D938D939C93D597C701B6012DEBE1
:106D500037E346E051E40E947B510E94154FF80151
:106D6000648F758F868F978FA0904A05B0904B05E2
:106D7000C0904C05D0904D05ABA6BCA6CDA6DEA616
:106D8000298D3A8D4B8D5C8D2FAB38AF49AF5AAF03
:106D900040914E0550914F056091500570915105FD
:106DA0004FA758AB69AB7AABCB01BA0120E030E01A
:106DB00040E05FE30E947B51162FE72E082FF92E4B
:106DC0006FA978AD89AD9AAD9F77212F3E2D402FC9
:106DD0005F2D0E94A950181664F0C601B50120E08D
:106DE00030E040E05FE30E947B51162FE72E082F32
:106DF000F92E8DE490E069A17AA1689FD001699F86
:106E0000B00D789FB00D1124A658BA4FFD01B2966F
:106E10009296CC90D180B280A380612F7E2D802F5E
:106E20009F2DF5012C2D3D2D4F2F5E2F0E94A64E3C
:106E300087FD04C01C2DED2C0B2DFA2C8D8D9E8D05
:106E4000AF8DB8A12B968CAF9DAFAEAFBFAF2B97D8
:106E500020915205309153054091540550915505AC
:106E60002FA338A749A75AA7CA01B90120E030E0EB
:106E700040E05FE30E947B51962E872E482E392EEC
:106E80002B966CAD7DAD8EAD9FAD2B979F77D401CA
:106E90002B2F3A2F442D532D0E94A95018168CF4F5
:106EA000612F7E2D802F9F2DD4012B2F3A2F442D23
:106EB000532D0E94A64E87FD04C0192DE82C042DE9
:106EC000F32C4BA15CA1423051050CF407C1609139
:106ED0004D0A70914E0A80914F0A9091500A27E115
:106EE00037EB41ED58E30E94A95018160CF0F6C09C
:106EF0006091510A7091520A8091530A9091540AFC
:106F00006BA37CA38DA39EA369897A898B899C89B5
:106F10002BA13CA14DA15EA10E94CC4D9B01AC01D7
:106F20000E947B51362E272E782E592E8091550A9D
:106F30009091560AA091570AB091580A60968CAF6A
:106F40009DAFAEAFBFAF60976D897E898F89988DF9
:106F500060962CAD3DAD4EAD5FAD60970E94CC4DBF
:106F60009B01AC010E947B51462E672E4C01B10162
:106F7000272F362F472D552DCA01B901242D362D27
:106F8000482D592D0E94CD4D0E94E8512B013C0106
:106F90006BA17CA18DA19EA19F7727E137EB41EDED
:106FA00058E30E94A95018169CF060966CAD7DAD18
:106FB0008EAD9FAD60979F7727E137EB41ED58E3AA
:106FC0000E94A950181624F0C12EDE2CB02EAF2C32
:106FD000C301B2012BA53CA54DA55EA50E94A950F9
:106FE0001816A4F46BA57CA58DA59EA5A3019201FE
:106FF0000E94AD4E9B01AC01F5016C2D7D2D8F2FB4
:107000009A2D0E947B516B01B82EA92E6FA978ADE5
:1070100089AD9AAD2091590A30915A0A40915B0A84
:1070200050915C0A0E94CC4D7B018C01E89417F9C9
:10703000C801B7012FA538A949A95AA90E94A9508A
:107040001816A4F46FA578A989A99AA9A80197018F
:107050000E94AD4E9B01AC01F5016C2D7D2D8F2F53
:107060009A2D0E947B516B01B82EA92E2B966CADE8
:107070007DAD8EAD9FAD2B9720915D0A30915E0A5C
:1070800040915F0A5091600A0E94CC4D7B018C01B7
:10709000E89417F9C801B7012FA138A549A55AA549
:1070A0000E94A9501816B4F46FA178A589A59AA5D5
:1070B000A80197010E94AD4E9B01AC01F5016C2D1A
:1070C0007D2D8F2F9A2D0E947B51162FE72E082F92
:1070D000F92E04C01C2DED2C0B2DFA2C8DE490E024
:1070E000A9A1BAA1A89F6001A99FD00CB89FD00CFC
:1070F0001124EAE7F5E0CE0EDF1E812F9E2DA02F92
:10710000BF2DF60182A793A7A4A7B5A722A933A9EB
:1071100044A955A95058CA01B9010E94CD4DD601C4
:107120009E962D913D914D915C91D1970E947B51FE
:107130009B01AC016BE077ED83E29BE30E94CC4DB9
:107140000E94E851B62EA72E982E892E612F7E2DF3
:10715000802F9F2DD501F4012B2F3A2F4F2F5E2F1B
:107160000E94A64E87FD04C01B2DEA2C092DF82C89
:107170008DE490E0E9A1FAA1E89F6001E99FD00CBD
:10718000F89FD00C11242AE735E0C20ED31E812FC0
:107190009E2DA02FBF2DF60186A397A3A0A7B1A770
:1071A00062A173A184A195A1D501F4012B2F3A2DE1
:1071B0004F2F582D0E94A64E181634F081E0D601AC
:1071C000D7968C93D79702C0F60117AA8DE490E06A
:1071D000A9A0BAA0A89EF001A99EF00DB89EF00D3E
:1071E0001124E658FA4F81E086ABA1E5BAE0FE0132
:1071F000719680E101900D928150E1F78DE490E06D
:10720000C9A0DAA0C89E8001C99E100DD89E100D9D
:10721000112406581A4FD8019296CD90DD90ED902A
:10722000FC909597C0924D0AD0924E0AE0924F0A78
:10723000F092500A96966D917D918D919C919997BF
:10724000A70196010E94AD4E4B015C016DEC7CECF8
:107250008CE49DE3A70196010E94AD4E6B017C0179
:10726000C801B501A401970186010E94DE292C9670
:10727000BFAD2C97B0934A0AABACBCACCDACDEAC86
:10728000A0926A05B0926B05C0926C05D0926D0514
:1072900023962CAD3DAD4EAD5FAD239720936E058B
:1072A00030936F05409370055093710527964CAD50
:1072B0005DAD6EAD7FAD279740937205509373051A
:1072C00060937405709375056BA97CA98DA99EA91F
:1072D0006093760570937705809378059093790590
:1072E0000E94D92DACD1C15BDF4F0FB6F894DEBF41
:1072F0000FBECDBFCF91DF911F910F91FF90EF9007
:10730000DF90CF90BF90AF909F908F907F906F90C5
:107310005F904F903F902F900895CF92DF92EF9221
:10732000FF920F931F93CF93DF938B017A01690133
:10733000FC01608171818281938120911E053091D1
:107340001F0540912005509121050E947B510E940C
:107350004B51CAE6D5E060936A0570936B05809344
:107360006C0590936D05F801608171818281938134
:107370002091220530912305409124055091250547
:107380000E947B510E944B518E010C5F1F4F6093F6
:107390006E05F801718382839383F70160817181A7
:1073A00082819381209126053091270540912805FF
:1073B000509129050E947B510E944B5148E0E42ED8
:1073C000F12CEC0EFD1E60937205F7017183828330
:1073D0009383F601608171818281938120912A05D6
:1073E00030912B0540912C0550912D050E947B5129
:1073F0000E944B51FE013C96609376057183828317
:107400009383CE01B801A7019F0171D780E090E07E
:10741000DC0180934D0A90934E0AA0934F0AB093DB
:10742000500A8093510A9093520AA093530AB09342
:10743000540A8093550A9093560AA093570AB09322
:10744000580A8093590A90935A0AA0935B0AB09302
:107450005C0A80935D0A90935E0AA0935F0AB093E2
:10746000600ADF91CF911F910F91FF90EF90DF9015
:10747000CF900895FC016081718182819381209178
:107480002A0530912B0540912C0550912D050E9425
:107490007B510E944B5160937605709377058093E2
:1074A00078059093790586E795E05DC780934C0A4F
:1074B00008958091950A882349F48091970A88233A
:1074C00029F48091990A882309F4AEC0E1E0FDE037
:1074D00007C09091C00095FFFCCF8093C600319605
:1074E00084918823B1F7E3E1FDE007C09091C000EB
:1074F00095FFFCCF8093C600319684918823B1F725
:107500008091950A882349F1EFE0FDE007C0909152
:10751000C00095FFFCCF8093C600319684918823EC
:10752000B1F76091630A7091640A8091650A909145
:10753000660A0E94484F20911E0530911F05409118
:107540002005509121050E94AD4EAB01BC0189E0A0
:1075500095E022E030E00E9495258091970A8823EB
:1075600049F1EBE0FDE007C09091C00095FFFCCF32
:107570008093C600319684918823B1F76091670AA1
:107580007091680A8091690A90916A0A0E94484F36
:107590002091220530912305409124055091250525
:1075A0000E94AD4EAB01BC0189E095E022E030E0E5
:1075B0000E9495258091990A882349F1E7E0FDE032
:1075C00007C09091C00095FFFCCF8093C600319614
:1075D00084918823B1F760916B0A70916C0A809155
:1075E0006D0A90916E0A0E94484F209126053091B5
:1075F000270540912805509129050E94AD4EAB0109
:10760000BC0189E095E022E030E00E949525809160
:10761000C00085FFFCCF8AE08093C6001092950AD7
:107620001092970A1092990A08951092950A109252
:10763000970A1092990A08958093FB010895EFE646
:10764000F0E080818260808308951F920F920FB6D0
:107650000F9211242F923F924F925F926F927F92DE
:107660008F929F92AF92BF92CF92DF92EF92FF9252
:107670000F931F932F933F934F935F936F937F933A
:107680008F939F93AF93BF93EF93FF93DF93CF932A
:1076900000D000D0CDB7DEB78091610A9091620A28
:1076A000009709F062C190914A0A80914B0A98179D
:1076B000A1F020914B0A30E08DE490E0289FF0018A
:1076C000299FF00D389FF00D1124E658FA4FDF0185
:1076D000A45BBF4F81E08C9302C0E0E0F0E0F09348
:1076E000620AE093610A309709F439C1DF01A45BB3
:1076F000BF4F81E08C931092A10A1092A20A1092BF
:10770000A30A1092A40A34AD25AD30939F0A2093AA
:10771000A00AC901692F782F27E26131720710F0A2
:1077200060E177E281E080939A0A6832710510F493
:1077300068E270E06852704038E060307307E0F053
:10774000872F90E0880F991F880F991F8F5F9A4F9E
:10775000FC01329645915491AA27659F9001649F40
:10776000210D3A1F06942A1F3A1F1124FC0145914E
:107770005491421B530B1FC0CB01969587958C7F6C
:107780008F5F964FFC01459154910296FC01259123
:107790003491E62FF0E0E770F0702E9FC0012F9F2C
:1077A000900D3E9F900D1124E3E096958795EA9504
:1077B000E1F7481B590B44365105A0F4E3EBF1E027
:1077C00006C09091C00095FFFCCF8093C6008191C8
:1077D0008823B9F789E095E04AE050E00E94D92477
:1077E00044E650E0CA01A0E0B0E080939B0A909389
:1077F0009C0AA0939D0AB0939E0A509389004093DF
:107800008800E091610AF091620A90AD81AD692F24
:10781000782F87E26131780710F060E177E281E04C
:1078200080939A0A6832710510F468E270E0685239
:107830007040E8E060307E07E0F0872F90E0880F2E
:10784000991F880F991F8F5F9A4FFC0132964591BF
:107850005491AA27659F9001649F210D3A1F0694B9
:107860002A1F3A1F1124FC0145915491421B530BCE
:107870001FC0CB01969587958C7F8F5F964FFC013B
:10788000459154910296FC0125913491E62FF0E048
:10789000E770F0702E9FC0012F9F900D3E9F900DBE
:1078A000112403E0969587950A95E1F7481B590B3B
:1078B00044365105A0F4E3EBF1E006C09091C0001E
:1078C00095FFFCCF8093C60081918823B9F789E0AA
:1078D00095E04AE050E00E94D92444E650E05093FD
:1078E000A60A4093A50AE091610AF091620A808994
:1078F0009189A289B389B695A79597958795B095F3
:10790000A095909581959F4FAF4FBF4F80937F0A71
:107910009093800AA093810AB093820A8093830A8D
:107920009093840AA093850AB093860A8093870A6D
:107930009093880AA093890AB0938A0A80938B0A4D
:1079400090938C0AA0938D0AB0938E0A10928F0A9E
:107950001092900A1092910A1092920A06C080ED3D
:1079600097E09093890080938800E091610AF091FC
:10797000620A309709F44AC480A18093930A80FF79
:107980003BC016988FEF8093F7018091FB0188230D
:10799000B9F123B1217031E0232759F18091940A84
:1079A000882339F180819181A281B381181619064B
:1079B0001A061B06F4F480916F0A9091700AA09148
:1079C000710AB091720A8093630A9093640AA0933B
:1079D000650AB093660A3093950A80899189A289D5
:1079E000B38980938F0A9093900AA093910AB093E1
:1079F000920A2093940A04C0169A81E08093F701BA
:107A00008091930A81FF3FC0149A8FEF8093F80111
:107A10008091FB018823D9F121E0199B02C020E06D
:107A20002FC08091960A882359F1E091610AF09164
:107A3000620A84819581A681B781181619061A06F3
:107A40001B06F4F48091730A9091740AA091750A50
:107A5000B091760A8093670A9093680AA093690AA6
:107A6000B0936A0A2093970A80899189A289B38981
:107A700080938F0A9093900AA093910AB093920AF0
:107A80002093960A04C0149881E08093F8018091B5
:107A9000930A82FF3FC046988FEF8093F90180914F
:107AA000FB018823D9F121E01A9B02C020E02FC0FE
:107AB0008091980A882359F1E091610AF091620A55
:107AC00080859185A285B385181619061A061B06AE
:107AD000F4F48091770A9091780AA091790AB09194
:107AE0007A0A80936B0A90936C0AA0936D0AB09304
:107AF0006E0A2093990A80899189A289B38980931B
:107B00008F0A9093900AA093910AB093920A2093BF
:107B1000980A04C0469A81E08093F9018091930A03
:107B200083FF03C045988FEF02C0459A81E08093A0
:107B3000FA0180919A0A282F30E03A832983209114
:107B40007F0A3091800A4091810A5091820A809187
:107B5000830A9091840AA091850AB091860AA09028
:107B6000870AB090880AC090890AD0908A0A6090EB
:107B70008B0A70908C0A80908D0A90908E0A1C82DD
:107B80001B8235C16091C00067FF19C02090C600FC
:107B9000E0910505F0910605BF016F5F7F4F6F779C
:107BA0007070E0900705F09008056E157F0539F0BC
:107BB000EB57FB4F20827093060560930505E0911B
:107BC000610AF091620AE080F180028113812E0D3A
:107BD0003F1D401F511F12161306140615060CF404
:107BE000159AE091610AF091620AE480F5800681BD
:107BF00017818E0D9F1DA01FB11F181619061A069A
:107C00001B060CF4139AE091610AF091620AE08479
:107C1000F18402851385AE0CBF1CC01ED11E1A1440
:107C20001B041C041D040CF4479AE091610AF091B6
:107C3000620AE484F584068517856E0C7F1C801E1D
:107C4000911E16141704180419040CF4179A12162E
:107C50001306140615061CF5E091610AF091620AFC
:107C6000E088F188028913892E193F09400B510BD6
:107C7000E0906F0AF090700A0091710A1091720AF8
:107C80006091F701E60EF11C011D111DE0926F0AD3
:107C9000F092700A0093710A1093720A15981816E0
:107CA00019061A061B061CF5E091610AF091620A9A
:107CB000E088F188028913898E199F09A00BB10B06
:107CC000E090730AF090740A0091750A1091760A98
:107CD0006091F801E60EF11C011D111DE092730A7E
:107CE000F092740A0093750A1093760A13981A1486
:107CF0001B041C041D041CF5E091610AF091620A4A
:107D0000E088F18802891389AE18BF08C00AD10A39
:107D1000E090770AF090780A0091790A10917A0A37
:107D20006091F901E60EF11C011D111DE092770A28
:107D3000F092780A0093790A10937A0A47981614F9
:107D40001704180419041CF5E091610AF091620A05
:107D5000E088F188028913896E187F08800A910AE9
:107D6000E0907B0AF0907C0A00917D0A10917E0AD7
:107D70006091FA01E60EF11C011D111DE0927B0AD3
:107D8000F0927C0A00937D0A10937E0A1798E09087
:107D90008F0AF090900A0091910A1091920A08942B
:107DA000E11CF11C011D111DE0928F0AF092900A56
:107DB0000093910A1093920A20908F0A3090900AB3
:107DC0004090910A5090920A6B817C816F5F7F4F47
:107DD0007C836B83E091610AF091620AE088F1880C
:107DE000028913892E143F044006510640F4EB81AA
:107DF000FC8169817A81E617F7070CF4C3CE2093E2
:107E00007F0A3093800A4093810A5093820A8093BC
:107E1000830A9093840AA093850AB093860AA0925D
:107E2000870AB092880AC092890AD0928A0A609220
:107E30008B0A70928C0A80928D0A90928E0A209101
:107E40008F0A3091900A4091910A5091920AE091E4
:107E5000610AF091620A84899589A689B789821797
:107E60009307A407B50708F4C8C020919B0A309176
:107E70009C0A40919D0A50919E0A648D758D868D55
:107E8000978DAA27279FB12D389F7001489FF00C2E
:107E9000479FE00CF11C289FB00DE11CFA1E379F94
:107EA000B00DE11CFA1E469FB00DE11CFA1E369F74
:107EB000B10DEA1EFA1EB695EA1EFA1E112424AD73
:107EC00035AD2E0D3F1D3093A00A20939F0A80AD43
:107ED00091ADA2ADB3AD40E050E082179307A40787
:107EE000B50720F49093A00A80939F0A90919F0A6F
:107EF0008091A00A692F782F87E26131780710F00E
:107F000060E177E281E080939A0A6832710510F4AB
:107F100068E270E068527040E8E060307E07E0F0B0
:107F2000872F90E0880F991F880F991F8F5F9A4FB6
:107F3000FC01329625913491AA27639FA001629F8C
:107F4000410D5A1F06944A1F5A1F1124FC01259106
:107F50003491241B350B1FC0CB01969587958C7FE0
:107F60008F5F964FFC01259134910296FC0145915B
:107F70005491E62FF0E0E770F0704E9FC0014F9FE4
:107F8000900D5E9F900D1124F3E096958795FA95DC
:107F9000E1F7281B390B24363105A0F4E3EBF1E0BF
:107FA00006C09091C00095FFFCCF8093C6008191E0
:107FB0008823B9F789E095E04AE050E00E94D9248F
:107FC00024E630E0309389002093880040E050E0C0
:107FD00080919B0A90919C0AA0919D0AB0919E0A63
:107FE000820F931FA41FB51F80939B0A90939C0A36
:107FF000A0939D0AB0939E0AE4C020918F0A30910D
:10800000900A4091910A5091920A808D918DA28D93
:10801000B38D82179307A407B50708F0CAC0209153
:10802000A10A3091A20A4091A30A5091A40A648D3A
:10803000758D868D978DAA27279FB12D389F70014A
:10804000489FF00C479FE00CF11C289FB00DE11CED
:10805000FA1E379FB00DE11CFA1E469FB00DE11CC1
:10806000FA1E369FB10DEA1EFA1EB695EA1EFA1EDA
:10807000112460919F0A7091A00A6E157F0538F453
:10808000DF01A05CBF4F6D917C91119702C06E190A
:108090007F09E05CFF4F80819181A281B3819B01C8
:1080A00040E050E0281739074A075B0708F4BC0195
:1080B000F7E261317F0710F060E177E281E08093C1
:1080C0009A0A6832710510F468E270E068527040F4
:1080D00028E060307207E0F0872F90E0880F991F4A
:1080E000880F991F8F5F9A4FFC013296259134912A
:1080F000AA27639FA001629F410D5A1F06944A1F41
:108100005A1F1124FC0125913491241B350B1FC0EB
:10811000CB01969587958C7F8F5F964FFC012591BB
:1081200034910296FC0145915491E62FF0E0E770FE
:10813000F0704E9FC0014F9F900D5E9F900D1124D7
:1081400043E0969587954A95E1F7281B390B24362D
:108150003105A0F4E3EBF1E006C09091C00095FF7B
:10816000FCCF8093C60081918823B9F789E095E020
:108170004AE050E00E94D92424E630E030938900A0
:108180002093880040E050E08091A10A9091A20ADB
:10819000A091A30AB091A40A820F931FA41FB51F38
:1081A0008093A10A9093A20AA093A30AB093A40A71
:1081B00008C08091A50A9091A60A909389008093A7
:1081C000880020918F0A3091900A4091910A509135
:1081D000920AE091610AF091620A80899189A289EC
:1081E000B389281739074A075B0780F01092620AA3
:1081F0001092610A90914A0A80914B0A981731F0C7
:1082000080914B0A8F5F8F7080934B0A2496DEBF5C
:10821000CDBFCF91DF91FF91EF91BF91AF919F9132
:108220008F917F916F915F914F913F912F911F910E
:108230000F91FF90EF90DF90CF90BF90AF909F9005
:108240008F907F906F905F904F903F902F900F9006
:108250000FBE0F901F9018950E9A0C9A3E9A3D9A59
:10826000529A529A529A529A2098289A2198299A68
:1082700022982A9A0D9A0B9A3F9A0F9AA1E8B0E099
:108280008C918F7E8C938C9188608C93E0E8F0E0E9
:1082900080818D7F808380818E7F808380818F73BA
:1082A000808380818F7C80838C91887F82608C9397
:1082B00080E090E49093890080938800109285007C
:1082C00010928400EFE6F0E080818260808381E09C
:1082D000B3D97894089590914A0A80914B0A9817DF
:1082E00029F092D281E00E948310F5CF0895CF93B8
:1082F000DF93EFB7F894EC0188819981AA81BB8163
:1083000080936F0A9093700AA093710AB093720AD7
:10831000EB0188819981AA81BB818093730A909334
:10832000740AA093750AB093760AEA01888199814C
:10833000AA81BB818093770A9093780AA093790AE7
:10834000B0937A0AE90188819981AA81BB818093DF
:108350007B0A90937C0AA0937D0AB0937E0AEFBFBC
:10836000DF91CF9108952FB7F894FC01808191811E
:10837000A281B38180937B0A90937C0AA0937D0AAB
:10838000B0937E0A2FBF08959FB7F894E82FF0E0CE
:10839000EE0FFF1FEE0FFF1FE159F54F20813181D6
:1083A000428153819FBFB901CA01089594DF5A9851
:1083B0005A985A985A98089560E070E08FE793E4CD
:1083C000209100023091010240910202509103027B
:1083D0000E94AD4E6093CE0A7093CF0A8093D00A6C
:1083E0009093D10A0895FC01ED54F54F808190E0FF
:1083F00008950F931F93CF93DF93EC01062F66230D
:1084000059F1E2E2FDE007C09091C00095FFFCCF7A
:108410008093C600319684918823B1F789E095E076
:10842000602F70E04AE050E00E94BC24EEECFEE0D9
:1084300007C09091C00095FFFCCF8093C600319695
:1084400084918823B1F78091C00085FFFCCF8AE03A
:108450008093C6000E945A10602F70E0660F771F4D
:10846000FB01E158FD4F80819181009709F45BC0C9
:108470006F577D4FFB01A081B18101E037C0A90199
:10848000440F551F440F551FFA013296E80FF91F8C
:10849000659174916C177D0744F5D9011197AA0F66
:1084A000BB1FAA0FBB1FFC01EA0FFB1F25913491D4
:1084B0001296A80FB91FFD0105911491840F951F05
:1084C000FC01A591B491A21BB30BC01BD10BAC9FB7
:1084D000C001AD9F900DBC9F900D1124601B710BCE
:1084E0000E946052620F731F19C00F5F202F30E08F
:1084F0002A173B070CF4C3CF2A173B0769F41197DF
:10850000AA0FBB1FAA0FBB1FA80FB91FFD018591A2
:108510009491682F792F02C060E070E020EF3FE374
:10852000261B370B16C0BE01882777FD8095982F34
:108530000E94484F2FE632E143E050E40E947B5115
:1085400020E030E040E851E40E947B510E94154F4A
:108550009B01C901DF91CF911F910F91089520E0F8
:1085600030E0D9011196AD01440F551F440F551F3E
:10857000FA01E154F24F65917491681779073CF55F
:10858000D901AA0FBB1FAA0FBB1FFD01E354F24F75
:1085900025913491A154B24FFD01A591B49143545A
:1085A000524FFA0145915491421B530BFC01EA1BB7
:1085B000FB0B4E9FC0014F9F900D5E9F900D1124AD
:1085C0006A1B7B0B0E946052620F731F12C0422F06
:1085D0004E5F9D01AC33B10509F0C3CF4D3339F483
:1085E000EDEAFEE085919491682F792F02C060E05A
:1085F00070E020EF3FE3261B370BC90108952F924F
:108600003F924F925F926F927F928F929F92AF9222
:10861000BF92CF92DF92EF92FF920F931F93CF936F
:10862000DF938C01E62E662359F1E2E2FDE007C0FC
:108630009091C00095FFFCCF8093C6003196849145
:108640008823B1F789E095E06E2D70E04AE050E0B4
:108650000E94BC24E1EBFEE007C09091C00095FFB2
:10866000FCCF8093C600319684918823B1F7809126
:10867000C00085FFFCCF8AE08093C6000E945A109C
:108680006E2D70E0660F771FFB01E158FD4F808172
:108690009181009709F488C0C0EFDFE3C01BD10BC4
:1086A0006F577D4FFB0160817181A1E060C09A012D
:1086B000220F331F220F331FFC01E20FF31FA5907F
:1086C000B490CA15DB050CF051C041505040440F26
:1086D000551F440F551FFA013296E80FF91F0591F7
:1086E0001491480F591FFA01859094902E5F3F4FC7
:1086F000280F391FF90165907490B801882777FD1C
:108700008095982F0E94484F1B012C01C819D90948
:10871000BE01882777FD8095982F0E94484F6B01F6
:108720007C01601A710AB301882777FD8095982F24
:108730000E94484F9B01AC01C701B6010E947B51CA
:108740007B018C01A818B908B501882777FD8095B1
:10875000982F0E94484F9B01AC01C801B7010E94AD
:10876000AD4E9B01AC01C201B10134C0AF5F4A2FD5
:1087700050E0461757070CF49ACF4617570769F58C
:10878000660F771F660F771F62507040680F791F62
:10879000FB01859194919C01B901882777FD809513
:1087A000982F0E94484F1DC0B801882777FD8095FB
:1087B000982F0E94484F20E030E04AEF5EE30E948D
:1087C0007B5120E030E040E85DE30E947B5120E0F7
:1087D00030E0A9010E94CD4D04C060E070E080E06F
:1087E00090E0DF91CF911F910F91FF90EF90DF907C
:1087F000CF90BF90AF909F908F907F906F905F9041
:108800004F903F902F9008952F923F924F925F92FA
:108810006F927F928F929F92AF92BF92CF92DF9290
:10882000EF92FF920F931F93DF93CF9300D000D06E
:10883000CDB7DEB78091B40A882309F4C8C18FB7D9
:10884000F8941092B40A8FBF8091AB0A9091AC0A51
:1088500060E0D5DE1B012C016091AF0A7091B00A77
:108860008091B10A9091B20AA20191010E94CC4D6F
:10887000162F072FF82EE92EA8019701852F942F88
:10888000A32FB22F8093D20A9093D30AA093D40A35
:10889000B093D50A652F742F832F922F20E030E0FC
:1088A00040E251E40E94A95018160CF42DC1A80111
:1088B0009701652F742F832F922F20E030E040E244
:1088C00051EC0E94A64E87FD1BC18091D60A8823D9
:1088D00009F008C1A8019701652F702F832F9E2DE5
:1088E0002091FC013091FD014091FE015091FF016A
:1088F0000E947B5169837A838B839C83472F382F17
:10890000292F862F942FA32FB22F8093DB0A9093C9
:10891000DC0AA093DD0AB093DE0AA8019701652F57
:10892000702F832F9E2D2091D70A3091D80A409125
:10893000D90A5091DA0A0E94CD4DD62EC72EB82EF4
:10894000A92EE090CA0AF090CB0A0091CC0A1091AF
:10895000CD0AA6019501652F742F832F922F2E2DFE
:108960003F2D402F512F0E94A64E87FF9FC08E2D76
:108970009F2DA02FB12F8093D70A9093D80AA09350
:10898000D90AB093DA0A6E2D7F2D802F912F209176
:1089900000023091010240910202509103020E94B4
:1089A0007B517B01082FB92E862F9F2DA02FBB2D29
:1089B0008093DF0A9093E00AA093E10AB093E20A61
:1089C000C201B1012091E30A3091E40A4091E50A25
:1089D0005091E60A0E94CC4D20910402309105028C
:1089E00040910602509107020E947B5120ED3CEC21
:1089F0004CE45DE30E947B513B014C016091E70A2E
:108A00007091E80A8091E90A9091EA0A23E333E33E
:108A100043E75FE30E947B519B01AC01C401B301BA
:108A20000E94CD4D162FD72EC82EA92E862F9D2DF4
:108A3000AC2DBA2D8093E70A9093E80AA093E90A37
:108A4000B093EA0A2092E30A3092E40A4092E50ADF
:108A50005092E60A59814A813B812C81652F742FFF
:108A6000832F922F2E2D3F2D402F5B2D0E94CD4D19
:108A7000212F3D2D4C2D5A2D0E94CC4D7B018C0178
:108A80007F2D912F20E030E0A9010E94A64E87FDA6
:108A900043C06E2D7F2D802F912F20E030E04FE7D7
:108AA00053E40E94A9501816DCF531C0E090CE0ABC
:108AB000F090CF0A0091D00A1091D10AA601950139
:108AC000652F742F832F922F2E2D3F2D402F512F46
:108AD0000E94A95018160CF44ACFED2CFC2C0B2D3B
:108AE0001A2D45CF80E090E0DC018093D70A909367
:108AF000D80AA093D90AB093DA0A1092D60AEACE1D
:108B000081E08093D60A08C081E08093D60AEE24E3
:108B1000FF240FE713E404C0EE24FF2400E010E07C
:108B20008091AB0A9091AC0A2091B50A3091B60AB7
:108B3000281739071CF01092B30A11C020910C02BB
:108B400030910D0282179307B4F76E2D7F2D802F81
:108B5000912F0E94154F759567956093B30A0E94F7
:108B600002222091EB0A3091EC0A4091ED0A5091DB
:108B7000EE0A621B730B840B950B683823E17207B6
:108B800020E0820720E0920710F10E940222609309
:108B9000EB0A7093EC0A8093ED0A9093EE0A8091B1
:108BA000AD0A9091AE0A1816190684F420910E02AF
:108BB00030910F02821793074CF42091A90A30914B
:108BC000AA0A8217930714F42C9A01C02C980F90CC
:108BD0000F900F900F90CF91DF911F910F91FF9009
:108BE000EF90DF90CF90BF90AF909F908F907F904D
:108BF0006F905F904F903F902F9008952F923F92EB
:108C00004F925F926F927F928F929F92AF92BF929C
:108C1000CF92DF92EF92FF920F931F93CF93DF9348
:108C2000C0EFDFE3C81BD90B80E090E0AC014F5FE1
:108C30005F4F9A01220F331F220F331FF901E354B4
:108C4000F24FA590B490CA15DB050CF04DC0880F0B
:108C5000991F880F991FFC01E154F24F059114915F
:108C60008354924FFC01859094902154324FF90126
:108C700065907490B801882777FD8095982F0E94A1
:108C8000484F1B012C01C819D909BE01882777FD5F
:108C90008095982F0E94484F6B017C01601A710AE1
:108CA000B301882777FD8095982F0E94484F9B013C
:108CB000AC01C701B6010E947B517B018C01A81851
:108CC000B908B501882777FD8095982F0E94484FF5
:108CD0009B01AC01C801B7010E94AD4E9B01AC01E4
:108CE000C201B1015AD718C0282F2E5FCA014C33D8
:108CF000510509F09BCF2D3359F4EFEAFEE0659161
:108D00007491882777FD8095982F0E94484F04C062
:108D100060E070E080E090E0DF91CF911F910F91D3
:108D2000FF90EF90DF90CF90BF90AF909F908F908B
:108D30007F906F905F904F903F902F90089580E0CC
:108D400090E0DC018093CA0A9093CB0AA093CC0AEE
:108D5000B093CD0A60E070E08FE793E420910002C9
:108D6000309101024091020250910302F6D76093C4
:108D7000CE0A7093CF0A8093D00A9093D10A239A97
:108D8000249A569A8EE061E070E00E94A32187ED5C
:108D900080937A00EEE7F0E010828081816080832A
:108DA0008081826080838081846080838081846010
:108DB000808380E888BDEEE6F0E080818460808377
:108DC0006AEF70E080E090E00E94382285E090E059
:108DD00060E00FDB9093B60A8093B50A83E191E0DF
:108DE00060E007DB90930D0280930C0286E990E02F
:108DF000B6DB90930F0280930E020895089580E0F1
:108E000090E060E0F6DA80E090E0DC018093AF0A69
:108E10009093B00AA093B10AB093B20A80E090E0B8
:108E20009EDB9093AA0A8093A90A1092A80A109236
:108E3000A70A1092B30A2B981092AA0A1092A90AB4
:108E40001092B40A1092AC0A1092AB0A1092B50AB2
:108E50001092AA0A1092A90A2C9808952F923F9274
:108E60004F925F926F927F928F929F92AF92BF923A
:108E7000CF92DF92EF92FF920F931F93DF93CF93E6
:108E8000CDB7DEB7E1970FB6F894DEBF0FBECDBF0A
:108E90006E877F87888B998B0E9402226A8B7B8BDF
:108EA0008C8B9D8BE7ECF1E006C09091C00095FFA4
:108EB000FCCF8093C60081918823B9F78091C000D0
:108EC00085FFFCCF8AE08093C60099DF8FE780930F
:108ED000B30AAA88BB88CC88DD88AA86BB86CC86E4
:108EE000DD86AE82BF82C886D9864FE7442E512CDC
:108EF000612C712C3FE7E32EF12C012D112D9924CB
:108F0000939420E030E0E9ECFFE0B490BCA2E4EC04
:108F1000FFE0C490CDA2EDEBFFE0D490DEA2E6EB43
:108F2000FFE044914FA3E0EBFFE0549158A7EAEA39
:108F3000FFE0849189A7EDE9FFE094919AA7E7E922
:108F4000FFE0A491ABA7E1E9FFE0B491BCA7EBE897
:108F5000FFE0A490ADA6ECE5FFE0B490BEA6E8E586
:108F6000FFE0C490CFA639AB28AB8091B40A882328
:108F700009F407C38FB7F8941092B40A8FBF809199
:108F8000AB0A9091AC0A60E03ADB69837A838B8309
:108F90009C835E894F89388D298D652F742F832F8F
:108FA000922FB981AA81DB80CC802B2F3A2F4D2DB7
:108FB0005C2D0E94A95018163CF0D980DE8A2A81C7
:108FC0002F8B3B81388FC98E5D81652F722D832D4C
:108FD000982DB981AA81DB80CC802B2F3A2F4D2D83
:108FE0005C2DB4D687FD05C049814D832A803D2C78
:108FF0008C2C992009F44CC059814A813B812C81E9
:10900000652F742F832F922FBE85AF85D888C9888E
:109010002B2F3A2F4D2D5C2D0E94A95018160CF0C5
:10902000B0C20E940222AA84BB84CC84DD846A1967
:109030007B098C099D09693823E1720720E08207CA
:1090400020E0920708F49DC2D801C7018419950950
:10905000A609B709B595A795979587958093B30A03
:109060000E9402226E837F8388879987DC01CB016F
:109070008A199B09AC09BD098E8F9F8FA8A3B9A33C
:109080009E859E8BAF85AF8BB889B88FE989E98FB4
:1090900059814A813B812C81652F742F832F922F18
:1090A000BE85AF85D888C9882B2F3A2F4D2D5C2DD2
:1090B0004DD687FF65C20E940222AE80BF80C88461
:1090C000D9846A197B098C099D09693823E17207E3
:1090D00020E0820720E0920708F452C20E94022298
:1090E0006A877B878C879D8748A959A941155105B7
:1090F00009F42DC2DC01CB018A199B09AC09BD0919
:10910000AE8CBF8CC8A0D9A0A80EB91ECA1EDB1E8B
:10911000AA8EBB8ECC8EDD8E2E8D3F8D48A159A19F
:10912000281B390B4A0B5B0BCA01B901A301920141
:109130000E944152A60195010E9495522E0D3F1D9D
:10914000401F511F2431310541055105ECF07901D3
:109150008A013CEEE316F104010511052CF0BBEE8B
:10916000EB2EF12C012D112D40E8E416F104010540
:109170001105ACF0AEEF4A2E512C612C712C4E181B
:109180005F08600A710A0DC0F4E1EF2EF12C012D89
:10919000112DE4E14E2E512C612C712C02C02701BF
:1091A00038018CA1E9ECFFE028A939A908C0909109
:1091B000C00095FFFCCF8093C60031968491882330
:1091C000B1F739AB28AB89E095E0B801A7012AE0F7
:1091D00030E00E948C248DA1E4ECFFE028A939A99D
:1091E00008C09091C00095FFFCCF8093C6003196D7
:1091F00084918823B1F739AB28AB89E095E0B301BE
:10920000A2012AE030E00E948C248EA1EDEBFFE069
:1092100028A939A908C09091C00095FFFCCF809380
:10922000C600319684918823B1F739AB28AB89E029
:1092300095E0FD814F2F522D632D782D22E030E0F7
:109240000E9495258FA1E6EBFFE028A939A908C067
:109250009091C00095FFFCCF8093C6003196849119
:109260008823B1F739AB28AB89E095E0FE89EF8917
:10927000388D298D4F2F5E2F632F722F22E030E023
:109280000E94952528A939A98091C00085FFFCCFAF
:1092900039AB28AB8AE08093C600233031050CF44B
:1092A00056C1C301B201F4D520E030E040E850E4FB
:1092B0000E947B515B016C015E894F89388D298D3D
:1092C000652F742F832F922FBD812B2F322D432D8D
:1092D000582D62D420ED3FE049E450E40E947B51D8
:1092E00020E030E040E05FE30E947B519B01AC0155
:1092F000C601B50132D5D62EC72EB82EA92E6A8D3D
:109300007B8D8C8D9D8DC4D520E030E04AE754E400
:1093100024D5962E872E382E292E88A5E0EBFFE047
:1093200028A939A908C09091C00095FFFCCF80936F
:10933000C600319684918823B1F739AB28AB89E018
:1093400095E0F60195014F2F5C2D632F7A2D22E0D9
:1093500030E00E94952589A5EAEAFFE028A939A90D
:1093600008C09091C00095FFFCCF8093C600319655
:1093700084918823B1F739AB28AB89E095E0F401FB
:1093800091014F2F582D632F722D22E030E00E9463
:10939000952528A939A98091C00085FFFCCF39AB5C
:1093A00028AB8AE08093C600A6019501652F7C2D2D
:1093B000832F9A2D2AE939E949E15FE39CD7D62E1C
:1093C000C72EB82EA92EA6019501652F742F832FC5
:1093D000922FD601F5012B2F3A2F4F2F5E2FDDD381
:1093E000D401F1012B2F382D4F2F522DB6D46D8380
:1093F0007A8F8AA39BA3A6019501652F742F832FD3
:10940000922FD401F1012B2F382D4F2F522D73D7CE
:1094100020E030E040E05EE36ED7962E872E382EB7
:10942000292E8AA5EDE9FFE028A939A908C0909165
:10943000C00095FFFCCF8093C600319684918823AD
:10944000B1F78091C00085FFFCCF39AB28AB8AE033
:109450008093C6008BA5E7E9FFE028A939A908C0D9
:109460009091C00095FFFCCF8093C6003196849107
:109470008823B1F739AB28AB89E095E0F601950177
:109480004F2F5C2D632F7A2D22E030E00E9495252E
:1094900028A939A98091C00085FFFCCF39AB28AB42
:1094A0008AE08093C6008CA5E1E9FFE028A939A9EC
:1094B00008C09091C00095FFFCCF8093C600319604
:1094C00084918823B1F739AB28AB89E095E0FD8121
:1094D000EA8D3AA12BA14F2F5E2F632F722F22E02E
:1094E00030E00E94952528A939A98091C00085FF08
:1094F000FCCF39AB28AB8AE08093C6008DA5EBE8A2
:10950000FFE028A939A908C09091C00095FFFCCFC1
:109510008093C600319684918823B1F739AB28AB8C
:1095200089E095E0F40191014F2F582D632F722DA2
:1095300022E030E00E94952528A939A98091C00039
:1095400085FFFCCF39AB28AB8AE08093C600D301FE
:10955000C2018E0D9F1DA01FB11FB595A7959795B0
:1095600087958093B30A88A999A9019699AB88AB8E
:109570009E859D832F84388889889924939401C07F
:1095800099245E854F8538892989652F742F832F0B
:10959000922F20E030E040EA51E4FFD29B01AC0181
:1095A000B981AA81DB80CC806B2F7A2F8D2D9C2DE9
:1095B000D0D5181694F4E2E6FFE007C09091C00001
:1095C00095FFFCCF8093C600319684918823B1F734
:1095D0008091C00085FFFCCFB5C00E940222AA88FE
:1095E000BB88CC88DD886A197B098C099D09613D9F
:1095F00027E0720720E0820720E0920708F44FC0BE
:109600000E9402226A8B7B8B8C8B9D8B8EA5ECE556
:10961000FFE028A939A908C09091C00095FFFCCFB0
:109620008093C600319684918823B1F739AB28AB7B
:109630008091AB0A9091AC0A60E00E94FF42AB01BE
:10964000BC0189E095E022E030E00E9495258FA5DD
:10965000E8E5FFE028A939A908C09091C00095FF6E
:10966000FCCF8093C600319684918823B1F739AB43
:1096700028AB80E090E00E94F341BC0189E095E0D6
:109680004AE050E00E94BC2428A939A98091C0007A
:1096900085FFFCCF39AB28AB8AE08093C6000E94DF
:1096A00002226A8F7B8F8C8F9D8F0E9402229B01EA
:1096B000AC018A8D9B8DAC8DBD8DAA84BB84CC847E
:1096C000DD848A199B09AC09BD09AE80BF80C884BE
:1096D000D9848A199B09AC09BD09820F931FA41F65
:1096E000B51F81382FE4920722E1A20720E0B207DC
:1096F00090F0EBE3FFE007C09091C00095FFFCCF36
:109700008093C600319684918823B1F78091C00080
:1097100085FFFCCF17C048A959A9463051050CF464
:1097200024CCEAEEFEE007C09091C00095FFFCCF8C
:109730008093C600319684918823B1F78091C00050
:1097400085FFFCCF8AE08093C600E1960FB6F894BF
:10975000DEBF0FBECDBFCF91DF911F910F91FF9064
:10976000EF90DF90CF90BF90AF909F908F907F90C1
:109770006F905F904F903F902F900895DF93CF931D
:109780000F92CDB7DEB789833ADB0E94A0216981B1
:10979000882379F5E2E2FDE007C09091C00095FFD3
:1097A000FCCF8093C600319684918823B1F789E07D
:1097B00095E070E04AE050E00E94BC248091C00037
:1097C00085FFFCCF8AE08093C600E0E9FDE007C09A
:1097D0009091C00095FFFCCF8093C6003196849194
:1097E0008823B1F78091C00085FFFCCF8AE0809389
:1097F000C6000F90CF91DF910895DF93CF930F9222
:10980000CDB7DEB78983FBDA0E94A0216981882366
:1098100079F5E2E2FDE007C09091C00095FFFCCF32
:109820008093C600319684918823B1F789E095E052
:1098300070E04AE050E00E94BC248091C00085FFA7
:10984000FCCF8AE08093C600E3E6FDE007C090917C
:10985000C00095FFFCCF8093C60031968491882389
:10986000B1F78091C00085FFFCCF8AE08093C600ED
:109870000F90CF91DF9108952C980E94A02188230A
:1098800009F5E2E2FDE007C09091C00095FFFCCF32
:109890008093C600319684918823B1F7E9E2FDE018
:1098A00007C09091C00095FFFCCF8093C600319611
:1098B00084918823B1F78091C00085FFFCCF8AE0B6
:1098C0008093C60008951F920F920FB60F92112435
:1098D0002F933F934F935F936F937F938F939F93B8
:1098E000AF93BF93EF93FF9380911002882331F4DD
:1098F0009091B30A9093B70A91112B9A9091B70A5D
:10990000891708F02B988F5F8F77809310028091D2
:10991000B80A833009F448C0843028F48130E1F07B
:109920008230C0F50DC0853009F466C0853008F47A
:1099300057C0863009F47CC0873009F0A6C084C0C7
:1099400010927B0080E480937C0080917A00806498
:1099500080937A0081E01BC02091780030917900DB
:1099600040E050E08091C50A9091C60AA091C70AD4
:10997000B091C80A820F931FA41FB51F8093C50A18
:109980009093C60AA093C70AB093C80A82E0809356
:10999000B80A7BC082E480937C0080917A00806466
:1099A00080937A0083E0F3CF2091780030917900A2
:1099B00040E050E08091B90A9091BA0AA091BB0AA8
:1099C000B091BC0A820F931FA41FB51F8093B90AE0
:1099D0009093BA0AA093BB0AB093BC0A84E0D7CF95
:1099E00010927B0081E480937C0080917A008064F7
:1099F00080937A0085E0CBCF209178003091790078
:109A000040E050E08091C10A9091C20AA091C30A3F
:109A1000B091C40A820F931FA41FB51F8093C10A7F
:109A20009093C20AA093C30AB093C40A86E0AFCF52
:109A300010927B0082E480937C0080917A008064A5
:109A400080937A0087E0A3CF20917800309179004D
:109A500040E050E08091BD0A9091BE0AA091BF0AFB
:109A6000B091C00A820F931FA41FB51F8093BD0A37
:109A70009093BE0AA093BF0AB093C00A1092B80A8E
:109A80008091C90A8F5F8093C90A8091C90A803189
:109A900008F471C02FEF3FE38091C50A9091C60A88
:109AA000A901481B590BCA015093AC0A4093AB0A59
:109AB0004091B90A5091BA0A241B350B3093AE0A73
:109AC0002093AD0A21E02093B40A1092C90A1092A3
:109AD000C50A1092C60A1092C70A1092C80A1092BC
:109AE000C10A1092C20A1092C30A1092C40A1092BC
:109AF000BD0A1092BE0A1092BF0A1092C00A1092BC
:109B0000B90A1092BA0A1092BB0A1092BC0A2091AC
:109B10000C0230910D028217930744F01092A80AAC
:109B20001092A70A80E02ADE0E9465212091AB0AEC
:109B30003091AC0A8091B50A9091B60A82179307CA
:109B400044F01092A80A1092A70A80E056DE0E9404
:109B500065212091AD0A3091AE0A80910E0290915C
:109B60000F02281739073CF01092AA0A1092A90A8E
:109B700083DE0E946521FF91EF91BF91AF919F918C
:109B80008F917F916F915F914F913F912F910F90A6
:109B90000FBE0F901F9018955058BB27AA270ED0C4
:109BA00076C23FD230F044D220F031F49F3F11F41E
:109BB0001EF40FC20EF4E095E7FBDCC1E92F89D259
:109BC00080F3BA17620773078407950718F071F4DA
:109BD0009EF5B8C20EF4E0950B2EBA2FA02D0B0106
:109BE000B90190010C01CA01A0011124FF27591BE2
:109BF00099F0593F50F4503E68F11A16F040A22FE8
:109C0000232F342F4427585FF3CF46953795279558
:109C1000A795F0405395C9F77EF41F16BA0B620B57
:109C2000730B840BBAF09150A1F0FF0FBB1F661F9E
:109C3000771F881FC2F70EC0BA0F621F731F841FE1
:109C400048F4879577956795B795F7959E3F08F007
:109C5000B3CF9395880F08F09927EE0F97958795C6
:109C60000895DFD158F080E891E009F49EEFE0D14B
:109C700028F040E851E059F45EEF09C0AAC162C281
:109C8000E92FE07826D268F3092E052AC1F32617BA
:109C900037074807590738F00E2E07F8E02569F016
:109CA000E025E0640AC0EF6307F8009407FADB01DF
:109CB000B9019D01DC01CA01AD01EF935DD0E7D18F
:109CC0000AD05F91552331F02BED3FE049E450FD80
:109CD00049EC63CF0895DF93DD27B92FBF7740E8C4
:109CE0005FE31616170648075B0710F4D92F96D2C4
:109CF0009F938F937F936F93A9D3E0E7F0E06CD1AC
:109D0000C6D12F913F914F915F9101D3DD2349F04F
:109D10009058A2EA2AED3FE049EC5FE3D0785D2756
:109D20004DDFDF91B4C1F7D180F09F3740F491113E
:109D30000EF409C260E070E080E89FE3089526F029
:109D40001B16611D711D811D1BC135C1EFD008F4AB
:109D500081E0089575D1E395ABC10CD098C168D16D
:109D600040F05FD130F021F45F3F19F003C1511191
:109D7000EAC12FC1AED198F39923C9F35523B1F3AA
:109D8000951B550BBB27AA2762177307840738F06A
:109D90009F5F5F4F220F331F441FAA1FA9F333D0C9
:109DA0000E2E3AF0E0E830D091505040E695001C7D
:109DB000CAF729D0FE2F27D0660F771F881FBB1F39
:109DC000261737074807AB07B0E809F0BB0B802D13
:109DD000BF01FF2793585F4F2AF09E3F510568F05F
:109DE000C9C0B1C15F3FECF3983EDCF3869577952F
:109DF0006795B795F7959F5FC9F7880F911D969561
:109E0000879597F90895E1E0660F771F881FBB1FBC
:109E1000621773078407BA0720F0621B730B840B69
:109E2000BA0BEE1F88F7E095089504D06894B1113D
:109E30008AC1089556D188F09F5790F0B92F99277D
:109E4000B751A0F0D1F0660F771F881F991F1AF045
:109E5000BA95C9F712C0B13081F074D1B1E008955C
:109E600071C1672F782F8827B85F39F0B93FCCF3DD
:109E7000869577956795B395D9F73EF4909580953B
:109E8000709561957F4F8F4F9F4F0895E89409C05B
:109E900097FB3EF490958095709561957F4F8F4F1D
:109EA0009F4F9923A9F0F92F96E9BB279395F69533
:109EB000879577956795B795F111F8CFFAF4BB0FB1
:109EC00011F460FF1BC06F5F7F4F8F4F9F4F16C015
:109ED000882311F096E911C0772321F09EE8872F9F
:109EE000762F05C0662371F096E8862F70E060E05B
:109EF0002AF09A95660F771F881FDAF7880F9695D4
:109F0000879597F9089507D180F09F3740F4911114
:109F10000EF019C160E070E080E89FEB089526F430
:109F20001B16611D711D811D2BC045C0990F0008B6
:109F3000550FAA0BE0E8FEEF16161706E807F9071B
:109F4000C0F012161306E407F50798F0621B730BB6
:109F5000840B950B39F40A2661F0232B242B252B37
:109F600021F408950A2609F4A140A6958FEF811DDA
:109F7000811D089597F99F6780E870E060E008957B
:109F8000882371F4772321F09850872B762F07C010
:109F9000662311F499270DC09051862B70E060E084
:109FA0002AF09A95660F771F881FDAF7880F969523
:109FB000879597F908959F3F31F0915020F4879548
:109FC00077956795B795880F911D9695879597F921
:109FD00008959FEF80EC0895DF93CF931F930F9325
:109FE000FF92EF92DF927B018C01689405C0DA2E1C
:109FF000EF018DD1FE01E894A59125913591459110
:10A000005591AEF3EF01DADDFE019701A801DA9474
:10A0100079F7DF90EF90FF900F911F91CF91DF9133
:10A02000089500240A9416161706180609060895BE
:10A0300000240A9412161306140605060895C9CFC3
:10A0400050D0E8F3E894E0E0BB279F57F0F02AED0A
:10A050003FE049EC06C0EE0FBB0F661F771F881F5D
:10A0600028F0B23A62077307840728F0B25A620BED
:10A07000730B840BE3959A9572F7803830F49A95B8
:10A08000BB0F661F771F881FD2F7904896CF092E07
:10A090000394000C11F4882352F0BB0F40F4BF2B43
:10A0A00011F460FF04C06F5F7F4F8F4F9F4F089583
:10A0B000EF93E0FF06C0A2EA2AED3FE049EC5FEB38
:10A0C0007DDDE5DF0F90039401FC9058EDE9F0E0B1
:10A0D000C7C157FD9058440F551F59F05F3F71F0AD
:10A0E0004795880F97FB991F61F09F3F79F08795FF
:10A0F0000895121613061406551FF2CF4695F1DF88
:10A1000008C0161617061806991FF1CF8695710517
:10A11000610508940895E5DFA0F0BEE7B91788F45B
:10A12000BB279F3860F41616B11D672F782F88273C
:10A13000985FF7CF869577956795B11D939596397A
:10A14000C8F30895E894BB2766277727CB0197F9D2
:10A150000895ECDE08F48FEF089563DF19F068DFEF
:10A1600009F037CF07CFB901CA0125CF9F775F77B5
:10A17000B0DF98F39923B9F35523B9F3FF27951767
:10A1800058F4E52FE91BED3070F75E3B10F0F1E479
:10A190001CC09034E0F40AC0E92FE51BED3028F72D
:10A1A0009E3B10F0F1E411C0503488F4F9EA8823A2
:10A1B0002AF09A95660F771F881FDAF744232AF052
:10A1C0005A95220F331F441FDAF79F1B5F1BFF9323
:10A1D0001F930F93FF92EF9279018A01BB27AB2F58
:10A1E0009B01AC0196D09701A801BF937B018C0124
:10A1F000AA27BA2FB901CA018CD0AF919701A80143
:10A20000EF90FF900F911F91D9DC41DFE1D04F918A
:10A2100040FF0895552747FD509509C09B01AC01AB
:10A2200060E070E080E89FE398CDA4CEC4CE59DF13
:10A23000E8F39923D9F3940F511DBBF3915050408B
:10A2400094F059F0882332F0660F771F881F9150E1
:10A250005040C1F79E3F510544F7880F911D9695D8
:10A26000879597F908955F3FACF0983E9CF0BB2727
:10A27000869577956795B79508F4B1609395C1F782
:10A28000BB0F58F711F460FFE8CF6F5F7F4F8F4F20
:10A290009F4FE3CF58CF25DF58F19E5758F1985183
:10A2A000A0F0E9F0983020F5092E9927660F771F66
:10A2B000881F991F0A94D1F712C0062E672F782F96
:10A2C0008827985F11F4000C07C0993FB4F3869576
:10A2D000779567959395D9F7611D711D811D3EF4A2
:10A2E00090958095709561957F4F8F4F9F4F089502
:10A2F000689429CF27CF0BD0CACE93DE28F098DE02
:10A3000018F0952309F036CE64CE11241CCFE1DE7F
:10A31000A0F3959FD1F3950F50E0551F629FF00178
:10A32000729FBB27F00DB11D639FAA27F00DB11DD1
:10A33000AA1F649F6627B00DA11D661F829F22275A
:10A34000B00DA11D621F739FB00DA11D621F839FE1
:10A35000A00D611D221F749F3327A00D611D231FB7
:10A36000849F600D211D822F762F6A2F11249F5705
:10A3700050408AF0E1F088234AF0EE0FFF1FBB1F28
:10A38000661F771F881F91505040A9F79E3F5105C7
:10A3900070F0F0CDD8CE5F3FECF3983EDCF38695BD
:10A3A00077956795B795F795E7959F5FC1F7FE2B72
:10A3B000880F911D9695879597F908959F9340DE94
:10A3C0000F9007FCEE5F74CE11F40EF402CEF3CDC5
:10A3D00088DED0F39923D9F3CEF39F57550B87FF2F
:10A3E00038D00024A0E640EA900180585695979511
:10A3F00028F4805C660F771F881F20F02617370728
:10A40000480730F4621B730B840B202931294A2B37
:10A41000A69517940794202531254A2758F7660FEB
:10A42000771F881F20F026173707480730F4620B84
:10A43000730B840B200D311D411DA09581F7B901CF
:10A44000842F9158880F9695879508959B01AC01AC
:10A4500052CF91505040660F771F881FD2F7089552
:10A460009F938F937F936F93FF93EF939B01AC0127
:10A4700042DFEF91FF91B0DD2F913F914F915F91BE
:10A480003ACF629FD001739FF001829FE00DF11DD2
:10A49000649FE00DF11D929FF00D839FF00D749F5E
:10A4A000F00D659FF00D9927729FB00DE11DF91F0A
:10A4B000639FB00DE11DF91FBD01CF011124089567
:10A4C00097FB092E07260AD077FD04D049D006D085
:10A4D00000201AF4709561957F4F0895F6F79095D6
:10A4E00081959F4F0895A1E21A2EAA1BBB1BFD0167
:10A4F0000DC0AA1FBB1FEE1FFF1FA217B307E40763
:10A50000F50720F0A21BB30BE40BF50B661F771FBA
:10A51000881F991F1A9469F760957095809590959A
:10A520009B01AC01BD01CF01089597FB092E0526C3
:10A530000ED057FD04D0D7DF0AD0001C38F4509558
:10A540004095309521953F4F4F4F5F4F0895F6F757
:10A5500090958095709561957F4F8F4F9F4F08958F
:10A56000AA1BBB1B51E107C0AA1FBB1FA617B70739
:10A5700010F0A61BB70B881F991F5A95A9F7809555
:10A580009095BC01CD010895EE0FFF1F0590F49149
:10A59000E02D0994A1E0B0E0EFECF2E576C55B01B7
:10A5A0006115710521F0DB018C9311969C93482F66
:10A5B000592F6A01F601E1906F018F018E2D90E015
:10A5C00080D20097B9F7FE2DFD3229F4D601ED9027
:10A5D0008D0121E007C0BE2DBB3219F4F601E190D8
:10A5E0008F0120E068010894C108D108C60161ED1F
:10A5F0007FE043E050E029836CD22981009709F580
:10A6000072E0E72EF12CE00EF11EC70164ED7FE051
:10A6100045E050E05ED22981009729F467E0E62EFC
:10A62000F12CE00EF11EA114B10421F0D501119618
:10A63000FC92EE9220FF0AC130E020E090E88FEF1C
:10A640000DC1C60169ED7FE043E050E0298341D2AE
:10A650002981009731F060E070E0CB016624772417
:10A660000AC0A114B10409F4F5C00E5F1F4FF50133
:10A6700011830083EFC03E2D30533A30A0F52260A5
:10A68000E22FF0E0AF014870507022FF07C0411583
:10A69000510571F50894611C711C2AC041155105C2
:10A6A00019F00894610871086B017C0152E0CC0C30
:10A6B000DD1CEE1CFF1C5A95D1F76C0D7D1D8E1D07
:10A6C0009F1D660F771F881F991F630F711D811DC6
:10A6D000911D6839F9E97F07F9E98F07F9E19F07CB
:10A6E00038F0246005C03E3F39F423FD3FC02860A8
:10A6F000D801ED908D01BFCF353311F03531B1F573
:10A70000F80131913D3211F4206102C03B3241F435
:10A71000D80111963C911197319642E050E002C069
:10A7200041E050E030533A3020F08F01041B150B0C
:10A730001DC040E050E0BCE040385B075CF4DA014B
:10A74000AA0FBB1FAA0FBB1F4A0F5B1F440F551F49
:10A75000430F511D319130538F013A3060F324FF84
:10A7600003C0509541955F4F640E751EC22EDD24C7
:10A7700021FF08C0A114B10429F001501040F501D7
:10A780001183008383DB7B018C01F3E0CF22DD2486
:10A7900033E0C316D10421F417FB109517F9109577
:10A7A000C801B70120E030E0A901D0DA882309F41C
:10A7B00048C077FE09C040EFC42E4FE0D42E7094FD
:10A7C00061947108739404C038E0C32E30E1D32E35
:10A7D00026E0822E912C90E2A92EB12C0EC0F6011B
:10A7E0002591359145915491C801B70184DDE62E3C
:10A7F000F72E082F192F6A187B086A147B047CF740
:10A80000B594A7940894810891088114910429F0C3
:10A810008CEF9FEFC80ED91EF0CFB701C801282FCB
:10A82000220F292F221F2F3F31F020E030E0A90115
:10A830008DDA882331F482E290E09093F40A8093D9
:10A84000F30A3E2D2F2D902F812F08C030E020E0FD
:10A8500090E803C030E020E090EC8FE7F901AC0114
:10A860006F2F722F852F942F2196EEE02AC42F92FE
:10A870003F924F925F927F928F929F92AF92BF9240
:10A88000CF92DF92EF92FF920F931F93CF93DF93BC
:10A890004B01EA016115710519F0FB018083918379
:10A8A000209739F09E01225030402332310508F0C4
:10A8B000F1C0A82EB92EF50111915F017F01812F02
:10A8C00090E0FFD00097B9F71D3229F4F5011191FE
:10A8D0007F0101E006C01B3219F4F50111917F01DF
:10A8E00000E0209719F0C031D105B9F4103381F49C
:10A8F000F7018081883711F0883551F4F701118113
:10A9000082E090E0E80EF91E0260C0E1D0E005C0F0
:10A91000209719F41033C1F422C0C830D105F9F0E2
:10A92000C930D10524F4C230D10509F507C0CA30B9
:10A93000D10551F0C031D105D1F426C0A12CB12CE4
:10A94000C12CF0E4DF2E25C0CAE0D0E0ECECAE2E46
:10A95000ECECBE2EECECCE2EECE0DE2E1AC0C8E005
:10A96000D0E0A12CB12CC12C70E1D72E12C09E01D9
:10A97000442737FD4095542F60E070E080E090E878
:10A98000B2DD59016A0105C0A12CB12CC12C68E0CF
:10A99000D62E40E060E070E0CB011E01442437FC7D
:10A9A0004094542C50ED752E710EE72DEA3070F066
:10A9B000212F21542A3118F439EC732E06C0212F8F
:10A9C00021562A3128F529EA722E710E272D30E002
:10A9D0002C173D07ECF447FD17C0A616B706C806AE
:10A9E000D90678F0A20191014CDD670D711D811D22
:10A9F000911D6130F0E07F07F0E08F07F0E89F07DE
:10AA000010F04FEF01C041E0F70111917F01CACF73
:10AA10008114910491F0442339F00894E108F1087D
:10AA2000F401F182E08209C001FF1BC097012250AE
:10AA30003040F4013183208314C047FF12C000FF6F
:10AA400005C060E070E080E090E804C06FEF7FEF49
:10AA50008FEF9FE722E230E03093F40A2093F30A6D
:10AA600016C000FF08C090958095709561957F4F46
:10AA70008F4F9F4F0CC097FF0AC082E290E09093E7
:10AA8000F40A8093F30A6FEF7FEF8FEF9FE79B014C
:10AA9000AC0103C020E030E0A901B901CA01DF9197
:10AAA000CF911F910F91FF90EF90DF90CF90BF90CB
:10AAB000AF909F908F907F905F904F903F902F909E
:10AAC000089591113BC2803219F089508550D0F71A
:10AAD0000895FB01DC014150504088F08D91813494
:10AAE0001CF08B350CF4805E659161341CF06B3585
:10AAF0000CF4605E861B611171F3990B0895881B3D
:10AB0000FCCFFC018191861721F08823D9F7992782
:10AB100008953197CF010895FB0151915523A9F074
:10AB2000BF01DC014D9145174111E1F759F4CD0109
:10AB30000190002049F04D9140154111C9F3FB01EE
:10AB40004111EFCF81E090E001970895AEE0B0E0D1
:10AB5000EBEAF5E5A4C20D891E8986E08C831A8391
:10AB600009838FEF9FE79E838D839E01275E3F4F72
:10AB7000CE0101966F89788DA90108D0EF81F88503
:10AB8000E00FF11F10822E96E4E0A5C2ACE0B0E029
:10AB9000EBECF5E576C26C011B018A01FC01178222
:10ABA0001682838181FFC4C12E010894411C511C6F
:10ABB000F6019381F10193FD859193FF81911F012E
:10ABC000882309F4B1C1853239F493FD859193FF4F
:10ABD00081911F01853221F490E0B601C8D1E8CF00
:10ABE000EE24FF2420E02032B0F48B3269F08C3266
:10ABF00028F4803251F0833271F40BC08D3239F079
:10AC0000803349F421602CC02260246029C0286070
:10AC100027C0206125C027FD2CC0382F30533A3083
:10AC200098F426FF08C08E2D880FE82EEE0CEE0C4F
:10AC3000E80EE30E15C08F2D880FF82EFF0CFF0CC9
:10AC4000F80EF30E20620CC08E3221F426FD6CC18A
:10AC5000206406C08C3611F4206802C0883649F49E
:10AC6000F10193FD859193FF81911F01882309F0E4
:10AC7000BACF982F9554933018F09052933028F40F
:10AC80000C5F1F4FFFE3F9830DC0833631F083372C
:10AC900071F0833509F05CC021C0F801808189839F
:10ACA0000E5F1F4F420171E0A72EB12C15C062E06C
:10ACB000662E712C600E711EF8018080918026FF37
:10ACC00003C06E2D70E002C06FEF7FEFC4012C87D0
:10ACD00043D15C0183012C852F7716C052E0652E8D
:10ACE000712C600E711EF8018080918026FF03C0D8
:10ACF0006E2D70E002C06FEF7FEFC4012C8721D171
:10AD00005C012C852068830123FD1EC007C080E202
:10AD100090E0B6012C872BD1FA942C858F2D90E0F2
:10AD2000A816B906A0F310C0F40127FD859127FFEE
:10AD300081914F0190E0B6012C8719D12C85F1103B
:10AD4000FA940894A108B108A114B10469F7E9C004
:10AD5000843611F0893641F527FF08C0F80160817B
:10AD60007181828193810C5F1F4F09C0F80160815E
:10AD70007181882777FD8095982F0E5F1F4F4FE6D2
:10AD8000B42EB22297FF09C0909580957095619579
:10AD90007F4F8F4F9F4FF0E8BF2AA2012AE030E09B
:10ADA00012D1782E741844C0853731F43FEEB32E9B
:10ADB000B2222AE030E025C099EFB92EB2228F36B8
:10ADC000C1F0803720F4883509F0AEC00DC080375F
:10ADD00021F0883709F0A8C002C020E1B22AB4FEF1
:10ADE0000BC084E0B82A08C0B4FE09C0E6E0BE2A61
:10ADF00006C028E030E005C020E130E002C020E1DC
:10AE000032E0B7FE08C0F8016081718182819381D0
:10AE10000C5F1F4F07C0F8016081718180E090E0F6
:10AE20000E5F1F4FA201CFD0782E7418FFE7BF220C
:10AE3000B6FE0BC02EEFB2227E1438F4B4FE07C06B
:10AE4000B2FC05C08FEEB82202C0A72C01C0AE2C08
:10AE50008B2D90E0B4FE0DC0FE01E70DF11D2081A9
:10AE6000203319F4E9EEBE2209C0A394B2FE06C055
:10AE700004C086789070009709F0A3948B2C9924D5
:10AE8000B3FC13C0B0FE0EC0AF1428F4E72CEF0CD7
:10AE9000EA18AF2C07C0E72C05C080E290E0B601AD
:10AEA00066D0A394AF14C8F304C0AF1410F4FA181A
:10AEB00001C0FF2484FE0EC080E390E0B60157D0AD
:10AEC00082FE1DC081FE03C088E590E010C088E7C7
:10AED00090E00DC0C40186789070009781F081FCED
:10AEE00002C080E201C08BE2B7FC8DE290E0B601C7
:10AEF0003ED005C080E390E0B60139D0EA947E14DC
:10AF0000C8F37A94F201E70DF11D808190E0B6015B
:10AF10002ED07720B1F705C080E290E0B60127D0AF
:10AF2000FA94FF20C9F744CEF6012681378102C08A
:10AF30002FEF3FEFC9012C96E2E1BFC09927882788
:10AF40000895FC010590615070400110D8F780957C
:10AF500090958E0F9F1F0895FC01615070400190E5
:10AF60000110D8F7809590958E0F9F1F08950F932D
:10AF70001F93CF93DF938C01EB018B8181FF1BC06B
:10AF800082FF0DC02E813F818C819D81281739075A
:10AF900064F4E881F9810193F983E88306C0E885C8
:10AFA000F985802F0995009731F48E819F81019654
:10AFB0009F838E8302C00FEF1FEFC801DF91CF91F7
:10AFC0001F910F910895FA01AA27283051F12031DD
:10AFD00081F1E8946F936E7F6E5F7F4F8F4F9F4F2D
:10AFE000AF4FB1E03ED0B4E03CD0670F781F891F6F
:10AFF0009A1FA11D680F791F8A1F911DA11D6A0F3D
:10B00000711D811D911DA11D20D009F468943F91EF
:10B010002AE0269F11243019305D3193DEF6CF01EE
:10B020000895462F4770405D4193B3E00FD0C9F7B4
:10B03000F6CF462F4F70405D4A3318F0495D31FD21
:10B040004052419302D0A9F7EACFB4E0A695979574
:10B05000879577956795BA95C9F70097610571054A
:10B0600008959B01AC010A2E069457954795379594
:10B070002795BA95C9F7620F731F841F951FA01DEE
:10B0800008952F923F924F925F926F927F928F928C
:10B090009F92AF92BF92CF92DF92EF92FF920F9367
:10B0A0001F93CF93DF93CDB7DEB7CA1BDB0B0FB671
:10B0B000F894DEBF0FBECDBF09942A88398848882E
:10B0C0005F846E847D848C849B84AA84B984C884C4
:10B0D000DF80EE80FD800C811B81AA81B981CE0FBB
:10B0E000D11D0FB6F894DEBF0FBECDBFED010895A0
:04B0F000F894FFCF02
:10B0F4005573696E672044656661756C7420736569
:10B104007474696E67733A004D3131300048200021
:10B114004C20002569206D696E2C202569207365FB
:10B1240063004D31303420496E76616C696420656A
:10B134007874727564657220004D31303520496E23
:10B1440076616C6964206578747275646572200038
:10B154004D31303920496E76616C696420657874AC
:10B16400727564657220003F006F6B0020703A00B6
:10B1740020693A0020643A0020633A005400496E82
:10B1840076616C69642065787472756465720041D7
:10B1940063746976652045787472756465723A20C3
:10B1A400002E00537465707261746520746F20689A
:10B1B400696768203A2000504944204175746F74CF
:10B1C400756E652073746172740000803B45008065
:10B1D4003B4500007043000000006400640060EA26
:10B1E40000000080BB44010101010101713DE841FF
:10B1F400A97E443E756089440000803FFF3FFF3FC5
:10B204000158595A45000001001A0019000A0000AB
:10B2140000FFFF1C001B000A000100FFFF170016BF
:10B22400000A000200FFFFFFFFFFFF04000E0018EA
:10B234000015000A000300000001000200020028BB
:10B2440023000028230000640000001027000000F1
:10B2540000FA430000FA430000A04000003442001A
:10B2640000A04214AE9F4200002045F6C81544BD1C
:04B274000D3D00008C
:00000001FF
